:020000040000FA
:1000000068EF3CF0F76A140FF66E000EF722090055
:10001000F55012000A4E494320696E6974206572DA
:1000200072200000F76A340FF66E000EF722090006
:10003000F5501200204E494320706B742065727297
:100040002000F76A520FF66E000EF7220900F550F5
:100050001200204E49432070747220657272200095
:10006000F76A700FF66E000EF7220900F5501200C5
:100070004E6F2064617974696D650D0A0000F76A3E
:100080008E0FF66E000EF7220900F55012000D0AD1
:1000900053657269616C206E756D3F200000F76AD0
:1000A000AE0FF66E000EF7220900F550120048540C
:1000B00054502F20323030204F4B0D0A0D0A4E6F16
:1000C00020576562207061676573210D0A00F76A29
:1000D000DE0FF66E000EF7220900F550120063687D
:1000E00065636B656400F76AF60FF66E000EF72223
:1000F0000900F550120070617373776F72642E6897
:10010000746D0000F76A140FF66E010EF7220900F5
:10011000F55012006572726F722E68746D00F76A86
:100120002E0FF66E010EF7220900F550120020285E
:10013000444843502900F76A460FF66E010EF72235
:100140000900F55012002028537461746963290076
:10015000F76A600FF66E010EF7220900F5501200E3
:1001600057656220536D61727420503138413639C1
:1001700039390000F76A840FF66E010EF722090084
:10018000F550120056657220312E30373100F76A73
:100190009E0FF66E010EF7220900F55012004B5328
:1001A0002D313137464D2D560000F76ABA0FF66EE5
:1001B000010EF7220900F55012004B532D31313555
:1001C000464D2D560000F76AD60FF66E010EF72247
:1001D0000900F55012004B5449204E6574776F7238
:1001E0006B730000F76AF40FF66E010EF722090038
:1001F000F55012000D0A44484350204950207363C3
:10020000616E6E696E670000F76A180FF66E020E77
:10021000F7220900F55012004B533131372D000001
:10022000F76A300FF66E020EF7220900F550120041
:100230004B533131352D0000F76A480FF66E020E30
:10024000F7220900F55012000D0A0D0A0000F76AA6
:100250005E0FF66E020EF7220900F5501200576588
:100260006220536D61727420503138413600F76A54
:100270007E0FF66E020EF7220900F5501200436F52
:100280006E6669672000F76A960FF66E020EF72217
:100290000900F55012000D0A0D0A495020616464EE
:1002A000723A2000F76AB40FF66E020EF7220900C8
:1002B000F55012000D0A4E65746D61736B3A2000A3
:1002C000F76AD00FF66E020EF7220900F550120001
:1002D0000D0A476174657761792049503A20000022
:1002E000F76AF00FF66E020EF7220900F5501200C1
:1002F0000D0A4D616320616464723A200000F76A60
:100300000E0FF66E030EF7220900F55012000D0ACB
:10031000393343343620436865636B00F76A2C0F2A
:10032000F66E030EF7220900F5501200204F4B2005
:100330002100F76A420FF66E030EF7220900F5500E
:100340001200204661696C6564202100F76A5C0F29
:10035000F66E030EF7220900F55012000D0A5254F2
:100360004C3830313920436865636B00F76A7C0F85
:10037000F66E030EF7220900F55012000D0A323412
:100380004C4332353620436865636B00010EEA6EDC
:10039000680EE96EEF50D8B4DBEF01F0060E016E87
:1003A000006A002EFED7012EFBD77B0E006E002EBA
:1003B000FED7EF2EF3D7000C01011E51E96E1F513D
:1003C000EA6E000123C1EFFF010E01011E25E96E57
:1003D000000E1F21EA6E000122C1EFFF020E010193
:1003E0001E25E96E000E1F21EA6E000121C1EFFFFC
:1003F000030E01011E25E96E000E1F21EA6E0001A9
:1004000020C1EFFF000C0101676B666B0001010169
:1004100066510508D8B003D000011EEF02F00001BC
:1004200066C1A9FFA69CA69EA680A85001016727C9
:1004300000010101662B000107EF02F00101671FB7
:100440006751016E0001000CA96A36C0A8FFA69C86
:10045000A69EA684F250006EF29E0F01550EA76E66
:10046000AA0EA76EA6820001A6B234EF02F0A694EF
:100470000050F212010EA96E37C0A8FFA69CA69EDE
:10048000A684F250006EF29E0F01550EA76EAA0EC2
:10049000A76EA6820001A6B24BEF02F0A694005010
:1004A000F212020EA96E1CC0A8FFA69CA69EA684EE
:1004B000F250006EF29E0F01550EA76EAA0EA76EA7
:1004C000A6820001A6B262EF02F0A6940050F212DA
:1004D000030EA96E1BC0A8FFA69CA69EA684F25080
:1004E000006EF29E0F01550EA76EAA0EA76EA68291
:1004F0000001A6B279EF02F0A6940050F212040EA9
:10050000A96E1AC0A8FFA69CA69EA684F250006EF3
:10051000F29E0F01550EA76EAA0EA76EA6820001CD
:10052000A6B290EF02F0A6940050F212050EA96E4A
:1005300019C0A8FFA69CA69EA684F250006EF29E4B
:100540000F01550EA76EAA0EA76EA6820001A6B2D5
:10055000A7EF02F0A6940050F212130EA96E24C069
:10056000A8FFA69CA69EA684F250006EF29E0F01E4
:10057000550EA76EAA0EA76EA6820001A6B2BEEF08
:1005800002F0A6940050F212140EA96E23C0A8FF28
:10059000A69CA69EA684F250006EF29E0F01550EF8
:1005A000A76EAA0EA76EA6820001A6B2D5EF02F032
:1005B000A6940050F212150EA96E22C0A8FFA69CA8
:1005C000A69EA684F250006EF29E0F01550EA76EF5
:1005D000AA0EA76EA6820001A6B2ECEF02F0A694C6
:1005E0000050F212160EA96E21C0A8FFA69CA69E6E
:1005F000A684F250006EF29E0F01550EA76EAA0E51
:10060000A76EA6820001A6B203EF03F0A6940050E5
:10061000F212170EA96E28C0A8FFA69CA69EA6845B
:10062000F250006EF29E0F01550EA76EAA0EA76E35
:10063000A6820001A6B21AEF03F0A6940050F212AF
:10064000180EA96E27C0A8FFA69CA69EA684F250ED
:10065000006EF29E0F01550EA76EAA0EA76EA6821F
:100660000001A6B231EF03F0A6940050F212190E69
:10067000A96E26C0A8FFA69CA69EA684F250006E76
:10068000F29E0F01550EA76EAA0EA76EA68200015C
:10069000A6B248EF03F0A6940050F2121A0EA96E0B
:1006A00025C0A8FFA69CA69EA684F250006EF29ECE
:1006B0000F01550EA76EAA0EA76EA6820001A6B264
:1006C0005FEF03F0A6940050F21203EC02F001C0B9
:1006D0001EF1060EA96E1EC1A8FFA69CA69EA684AA
:1006E000F250006EF29E0F01550EA76EAA0EA76E75
:1006F000A6820001A6B27AEF03F0A6940050F2128F
:10070000000C899289948996800E01015A6F090E16
:100710005B6F010E5C6F000101015C510408D8B0F1
:1007200003D000019FEF03F00001D89001015A3778
:100730005B37000101015C2B00018CEF03F089861F
:10074000020E0101686F0001C6EC01F0010E01010B
:100750005C6F000101015C510A08D8B003D00001B0
:10076000C8EF03F00001D89001015A375B37D8A0D9
:1007700003D00001C0EF03F000018992C1EF03F044
:1007800089828984899401015C2B0001AAEF03F01E
:100790008992020E0101686F0001C6EC01F0899692
:1007A000080E006E002EFED789848994000C01018A
:1007B0006235636F6337FC0E63176135686F6837A6
:1007C000FC0E68176239006E00320032030E00160C
:1007D00000506811646F6035686F6837FC0E6817E9
:1007E0006139006E00320032030E001600506811AD
:1007F000656F050E666F010E676F0001010167519D
:100800000508D8B003D0000113EF04F00001D89020
:100810000101633764376537663700010101672BD3
:100820000001FEEF03F08986020E0101686F0001EE
:10083000C6EC01F08980010E0101676F0001010122
:1008400067511908D8B003D000013FEF04F0000150
:10085000D89001016337643765376637D8A003D075
:10086000000137EF04F00001899238EF04F089822B
:10087000898489940101672B00011FEF04F089929C
:100880008996030E006E002EFED789848994030E8C
:10089000006E002EFED7898689848994000E80B070
:1008A000010E0108D8B44CEF04F0020E0101686F8C
:1008B0000001C6EC01F08996080E006E002EFED7EE
:1008C00089848994320E0101686F0001C6EC01F041
:1008D000000C020EA96E5AC1A8FFA69CA69EA68473
:1008E000F250006EF29E0F01550EA76EAA0EA76E73
:1008F000A6820001A6B27AEF04F0A6940050F2128C
:10090000030EA96E5BC1A8FFA69CA69EA684F2500A
:10091000006EF29E0F01550EA76EAA0EA76EA6825C
:100920000001A6B291EF04F0A6940050F212040E5A
:10093000A96E5CC1A8FFA69CA69EA684F250006E7C
:10094000F29E0F01550EA76EAA0EA76EA682000199
:10095000A6B2A8EF04F0A6940050F212050EA96EFC
:100960005DC1A8FFA69CA69EA684F250006EF29ED2
:100970000F01550EA76EAA0EA76EA6820001A6B2A1
:10098000BFEF04F0A6940050F21203EC02F001C095
:1009900066F1060EA96E66C1A8FFA69CA69EA68457
:1009A000F250006EF29E0F01550EA76EAA0EA76EB2
:1009B000A6820001A6B2DAEF04F0A6940050F2126B
:1009C000130EA96E5EC1A8FFA69CA69EA684F25037
:1009D000006EF29E0F01550EA76EAA0EA76EA6829C
:1009E0000001A6B2F1EF04F0A6940050F212140E2A
:1009F000A96E5FC1A8FFA69CA69EA684F250006EB9
:100A0000F29E0F01550EA76EAA0EA76EA6820001D8
:100A1000A6B208EF05F0A6940050F212150EA96ECA
:100A200060C1A8FFA69CA69EA684F250006EF29E0E
:100A30000F01550EA76EAA0EA76EA6820001A6B2E0
:100A40001FEF05F0A6940050F212160EA96E61C1B8
:100A5000A8FFA69CA69EA684F250006EF29E0F01EF
:100A6000550EA76EAA0EA76EA6820001A6B236EF9B
:100A700005F0A6940050F212170EA96E62C1A8FFED
:100A8000A69CA69EA684F250006EF29E0F01550E03
:100A9000A76EAA0EA76EA6820001A6B24DEF05F0C2
:100AA000A6940050F212180EA96E63C1A8FFA69C6E
:100AB000A69EA684F250006EF29E0F01550EA76E00
:100AC000AA0EA76EA6820001A6B264EF05F0A69456
:100AD0000050F212190EA96E64C1A8FFA69CA69E32
:100AE000A684F250006EF29E0F01550EA76EAA0E5C
:100AF000A76EA6820001A6B27BEF05F0A694005077
:100B0000F2121A0EA96E65C1A8FFA69CA69EA68425
:100B1000F250006EF29E0F01550EA76EAA0EA76E40
:100B2000A6820001A6B292EF05F0A6940050F21240
:100B300035EF07F0010E926E81EC03F00101606B5E
:100B4000410E616F540E626F0001D7EC03F0130E7B
:100B50000101596F0001010159512208D8B003D099
:100B60000001C3EF05F0000159C160F1FF0E010162
:100B7000616F040E626F0001D7EC03F00101592B85
:100B80000001ABEF05F0140E0101606FFF0E616F05
:100B9000FF0E626F0001D7EC03F0230E0101596FC5
:100BA0000001010159513F08D8B003D00001E7EF1F
:100BB00005F0000159C160F10101616B626B000138
:100BC000D7EC03F00101592B0001D1EF05F0010E24
:100BD0000101596F0001010159510908D8B003D032
:100BE000000103EF06F0000159C160F1840E01011C
:100BF000616F4F0E626F0001D7EC03F00101592BBA
:100C00000001EBEF05F0030E0101606F840E616FD0
:100C1000410E626F0001D7EC03F0080E0101606F16
:100C2000C40E616F4D0E626F0001D7EC03F00A0E27
:100C30000101606F590E616F020E626F0001D7EC07
:100C400003F00B0E0101606F800E616F626B00019B
:100C5000D7EC03F00C0E0101606FFA0E616F500EBD
:100C6000626F0001D7EC03F00D0E0101606FFA0E08
:100C7000616F500E626F0001D7EC03F00E0E0101A0
:100C8000606F550E616F626B0001D7EC03F00F0EC1
:100C90000101606F550E616F626B0001D7EC03F0CC
:100CA000100E0101606F300E616F626B0001D7ECB6
:100CB00003F0110E0101606FFF0E616F626B0001A6
:100CC000D7EC03F0120E0101606F360E616F626B9C
:100CD0000001D7EC03F02C0E0101606FD00E616FA4
:100CE000626B0001D7EC03F02D0E0101606F450E21
:100CF000616F560E626F0001D7EC03F00101596B72
:100D00000001010159510708D8B003D00001AAEF32
:100D100006F000010A0E010159255A6F00015AC15F
:100D2000A9FFA86AA69CA69EA684F250006EF29E19
:100D30000F01550EA76EAA0EA76EA6820001A6B2DD
:100D40009FEF06F0A6940050F2120101592B00010A
:100D500081EF06F00A0EA96E310EA86EA69CA69E23
:100D6000A684F250006EF29E0F01550EA76EAA0ED9
:100D7000A76EA6820001A6B2BBEF06F0A6940050B3
:100D8000F2120B0EA96E320EA86EA69CA69EA68429
:100D9000F250006EF29E0F01550EA76EAA0EA76EBE
:100DA000A6820001A6B2D2EF06F0A6940050F2127D
:100DB0000C0EA96E330EA86EA69CA69EA684F250B9
:100DC000006EF29E0F01550EA76EAA0EA76EA682A8
:100DD0000001A6B2E9EF06F0A6940050F212080E48
:100DE000A96EA86AA69CA69EA684F250006EF29EEA
:100DF0000F01550EA76EAA0EA76EA6820001A6B21D
:100E0000FFEF06F0A6940050F212090EA96E020E32
:100E1000A86EA69CA69EA684F250006EF29E0F01BC
:100E2000550EA76EAA0EA76EA6820001A6B216EFF7
:100E300007F0A6940050F212C00E01015A6FA80EDE
:100E40005B6F5C6B020E5D6FFF0E5E6FFF0E5F6F80
:100E5000FF0E606F616BC00E626FA80E636F646BF4
:100E6000010E656F000169EF04F0000C25C103F06D
:100E700001012451E96E000103C0EAFFECCF03F049
:100E8000ED52EF50105C0101286F03501158296F8B
:100E900026512711D8A403D0000165EF07F0000107
:100EA00001012751295DD8B003D0000176EF07F08A
:100EB0000001D8A465EF07F001012651285DD8B0E4
:100EC00003D0000176EF07F0000125C103F0010116
:100ED0002451E96E000103C0EAFF11C0ECFFED529E
:100EE00010C0EFFF010E016E78EF07F0000E016EEB
:100EF000000C78C181FF79C183FF000E956E84924A
:100F000000008482FF0E956E000C0E0E0101752705
:100F1000400E7623070E786F400E796F000179EC52
:100F200007F0080E0101786F000175C179F179ECC5
:100F300007F076C177F1090E0101786F000177C1E2
:100F400079F179EC07F0010E6C6E000CFF0E956ED6
:100F500075C181FF849083CF76F184800101765141
:100F6000016E0001000C0101736B000171C074F18E
:100F700001017453D8B403D00001C2EF07F000019F
:100F800020EF08F001017451010B7427070E786FF0
:100F9000400E796F000179EC07F00A0E0101786FBD
:100FA000000174C179F179EC07F00B0E0101786F43
:100FB000796B000179EC07F00101786B120E796F03
:100FC000000179EC07F0100E816E000E956E0101A4
:100FD00074517407000AD8A403D0000101EF08F08F
:100FE000000101017351732B720FE96EEA6AD8B0E8
:100FF000EA2AEF50836E8492000084820001E7EFBA
:1010000007F0FF0E956EFF0E0101746F00010101E4
:101010007453D8A403D0000120EF08F00001070E9C
:101020000101756F0001A6EC07F00150400B000AAA
:10103000D8A420EF08F001017407000107EF08F0C1
:10104000000C7152D8B43AEF08F06C52D8A437EFC4
:1010500008F071506F5C0101736F000E7058746F6F
:10106000000174C176F173C175F185EC07F0B3EC42
:1010700007F0716A6E50705CD8A04BEF08F0D8A4EE
:1010800047EF08F06F506D5CD8B04BEF08F070C0C0
:101090006EF06FC06DF0000C29A061EF08F0010147
:1010A00073512B2673512B5CD8A003D000015FEF46
:1010B00008F000012A2AD8A45FEF08F02B2A71EF6C
:1010C00008F0010173512A2673512A5CD8A003D07D
:1010D000000171EF08F000012B2AD8A471EF08F08D
:1010E0002A2A2970000C70500408D8B085EF08F047
:1010F000FF0AD8A481EF08F06F50E908D8B085EF57
:1011000008F0000E016E9EEF08F071501F08D8B075
:101110008CEF08F021EC08F07150712A720FE96E23
:10112000EA6AD8B0EA2A72C1EFFF6F2AD8B4702AEF
:1011300072C173F14CEC08F0010E016E000C29A68F
:10114000B7EF08F0010171510A08D8B403D00001CB
:10115000B0EF08F000010D0E9EA8ACEF08F0AD6EE8
:101160000101715100019EA8B3EF08F0AD6E29A8EE
:10117000BEEF08F071C172F173EC08F0000CA96ABF
:10118000A69CA69EA680A850366E010EA96EA69CAF
:10119000A69EA680A850376E020EA96EA69CA69E9B
:1011A000A680A8501C6E030EA96EA69CA69EA680C3
:1011B000A8501B6E040EA96EA69CA69EA680A850E1
:1011C0001A6E050EA96EA69CA69EA680A850196E42
:1011D000130EA96EA69CA69EA680A850246E140E7F
:1011E000A96EA69CA69EA680A850236E150EA96E79
:1011F000A69CA69EA680A850226E160EA96EA69C3E
:10120000A69EA680A850216E170EA96EA69CA69E2B
:10121000A680A850286E180EA96EA69CA69EA68031
:10122000A850276E190EA96EA69CA69EA680A8504F
:10123000266E1A0EA96EA69CA69EA680A850256EA4
:10124000060EA96EA69CA69EA680A85001011C6F42
:10125000000103EC02F001011C51015CD8A403D091
:10126000000137EF09F00001000E38EF09F0010E20
:10127000016E000C3A50010174273B5075237551E3
:101280005E08D8A003D0000152EF09F0000101016F
:101290007451016EE70E7525036E0150746F0001E5
:1012A00003C075F1070E0101786F400E796F0001E0
:1012B00079EC07F0080E0101786F000174C179F133
:1012C00079EC07F075C176F1090E0101786F000124
:1012D00076C179F179EC07F06C6A000C416A41C083
:1012E00040F03F6A40C03EF0149C299A0101756BA2
:1012F000746B00013AEC09F0000C9EAA8EEF09F025
:10130000ABB48AEF09F0ABB28AEF09F0010E016EBF
:1013100090EF09F0AB98AECF24F1AB88000E016ED0
:10132000DCEF09F001011A51CF5C196F19517908EE
:10133000D8A003D00001A9EF09F00001102AD8B409
:10134000112A7A0E01011A27010E016E0001ABEF7E
:1013500009F0000E016EB0EF09F0040092EF09F001
:10136000000C9EBACBEF09F0ABB4BAEF09F0ABA218
:10137000CBEF09F0ABB4C0EF09F0ABA2C8EF09F0B6
:10138000AB98AECF24F1AB88000E016ECDEF09F023
:101390000400B1EF09F0AE50016E0CEF0AF001014C
:1013A000206B010E256F210E246F276B266B000129
:1013B00036EC07F07DEF09F00152D8A40AEF0AF0ED
:1013C00001011E511F11D8A403D0000106EF0AF03D
:1013D0000001010E0101256F210E246F00011FC1C4
:1013E00027F11EC126F136EC07F00152D8B406EF02
:1013F0000AF0420E01012025E96EEA6AD8B0EA2A15
:10140000EF6A2051016E0001B4EF0AF0ADEC09F073
:10141000DAEF09F0B1EF09F001C023F10101235126
:101420001F08D8A003D0000120EF0AF0000101013D
:1014300023517F08D8B403D000017CEF0AF00001EB
:10144000010123511B08D8B403D0000130EF0AF08A
:1014500000010101206B0001A2EF0AF07AEF0AF00F
:10146000010123510D08D8B403D000014EEF0AF05A
:10147000000101011E511F11D8A403D000014AEF41
:101480000AF0000101012053D8A403D000014CEF61
:101490000AF00001A2EF0AF07AEF0AF001012351ED
:1014A0000808D8A403D0000160EF0AF00001010190
:1014B00023517F08D8B403D000017AEF0AF000016D
:1014C00001012053D8A403D000017AEF0AF00001F3
:1014D00001012007080E00019EA86CEF0AF0AD6E16
:1014E000200E9EA871EF0AF0AD6E080E9EA876EF52
:1014F0000AF0AD6EA0EF0AF0010120512808D8B023
:1015000003D00001A0EF0AF0000101012051202BBF
:10151000420FE96EEA6AD8B0EA2A000123C1EFFF60
:1015200001011E511F11D8B403D00001A0EF0AF031
:1015300000010101235100019EA89CEF0AF0AD6E4D
:10154000DAEF09F0420E01012025E96EEA6AD8B00F
:10155000EA2AEF6A3D6A000120C13CF03CC040F03D
:1015600001012051016E0001B6EF0CF0010174532E
:10157000D8B403D00001C0EF0AF00001F9EF0AF07F
:10158000070E0101786F400E796F000179EC07F0CA
:101590000A0E0101786F000174C179F179EC07F04E
:1015A0000B0E0101786F796B000179EC07F00101F6
:1015B000786B0A0E796F000179EC07F0100E816EDE
:1015C000FF0E956E010174517407000AD8A403D070
:1015D0000001F9EF0AF0000184904050402A420FC8
:1015E000E96EEA6AD8B0EA2A83CFEFFF8480E2EF9F
:1015F0000AF0000C415001016E5DD8A003D000013B
:101600002EEF0BF000016EC170F14050415CD8B07C
:101610002AEF0BF001017051702B420F016E036A2B
:10162000D8B0032A0150756F000103C076F1415014
:10163000412A420FE96EEA6AD8B0EA2AEF50010166
:10164000786F000176C1EAFF75C1E9FF78C1EFFF4D
:1016500005EF0BF070C140F06EC141F03E503C5CB4
:101660000101726F3F503D58736F7353D8B403D06C
:1016700000014CEF0BF0000101016F51725DD8A029
:1016800003D000014CEF0BF0000173C103F0010126
:10169000725100014FEF0BF001016F510001010188
:1016A0006F6F2A0ED88040546F5DD8A403D000011C
:1016B00065EF0BF0D8B003D0000165EF0BF000012F
:1016C0002A0ED880405468EF0BF001016F510001E1
:1016D00001016F6F00016FC171F101017153D8A455
:1016E00003D0000183EF0BF000016C52D8B47FEF00
:1016F0000BF03FC075F13EC074F13AEC09F06FC1D8
:1017000074F1B6EC0AF001016F51016E0001000C9A
:101710004050415CD8A095EF0BF00A0E01016E6FAE
:101720002A0E6F6F0001FAEC0AF04050415CD8A01D
:101730009EEF0BF0000E016EC1EF0BF04150412AFD
:10174000420FE96EEA6AD8B0EA2AEF5001016D6FE4
:101750003E2AD8B43F2A29AA03D00001B5EF0BF0E6
:1017600000016DC173F14CEC08F06CC103F0010194
:101770006B51E96E000103C0EAFF6DC1EFFF010E7E
:10178000016E000C4152D8B4DCEF0BF03E503F101C
:10179000D8B4DCEF0BF04106420E4124E96EEA6A50
:1017A000D8B0EA2A24C1EFFF3E50D8B43F063E0627
:1017B000010E016EDEEF0BF0000E016E76EF0CF005
:1017C0000101206B216B236B0001010E01016C6F85
:1017D000220E6B6F000188EC0BF00152D8B47AEF47
:1017E0000CF0010122512F08D8A003D000011CEFFA
:1017F0000CF00001010122513908D8B003D00001DA
:101800001CEF0CF000010101232B300E225F20356C
:10181000246F2135256F2437253724372537243782
:101820002537F00E241722512425206F000E252184
:10183000216F000178EF0CF0010122514008D8A07F
:1018400003D0000147EF0CF00001010122514608CE
:10185000D8B003D0000147EF0CF000010101232BA9
:10186000370E225F2035246F2135256F2437253729
:101870002437253724372537F00E24172251242505
:10188000206F000E2521216F000178EF0CF001017F
:1018900022516008D8A003D0000172EF0CF00001C3
:1018A000010122516608D8B003D0000172EF0CF09C
:1018B00000010101232B570E225F2035246F2135B3
:1018C000256F243725372437253724372537F00E61
:1018D000241722512425206F000E2521216F00019D
:1018E00078EF0CF022C124F1C2EF0BF07AEF0CF08C
:1018F000E5EF0BF01FC103F001011E51E96E00017D
:1019000003C0EAFF21C1ECFFED5220C1EFFF01014E
:101910002353D8B403D0000192EF0CF00001000E65
:1019200093EF0CF0010E016EC2EF0CF001011E6B83
:10193000000101011E5100013FEC00F001011E2BCE
:1019400000019EA8A1EF0CF0AD6E0E0E01011E5D10
:10195000D8B403D0000199EF0CF000016EEC09F04F
:1019600001011F6B1E6B0001CFEF09F00152D8B4CB
:10197000CAEF0CF0010E01011F6F1C0E1E6F00015B
:10198000E0EF0BF00152D8B4CAEF0CF01DC136F0F5
:101990001CC137F00D0E9EA8CBEF0CF0AD6E0A0EF9
:1019A0009EA8D0EF0CF0AD6E01011F6B190E1E6FDB
:1019B000C00E206FA80E216F226B020E236F000154
:1019C000DCEC01F001011F6B210E1E6FFF0E206F7A
:1019D000FF0E216FFF0E226F236B0001DCEC01F084
:1019E00001011F6B250E1E6FC00E206FA80E216F08
:1019F000226B010E236F0001DCEC01F024EC02F0FD
:101A0000010E016E14EF3EF001015C6B5D6B5B3506
:101A10005E6F5E37FC0E5E17060E5F6F010E606F25
:101A20000001010160510508D8B003D0000126EF84
:101A30000DF00001D89001015C375D375E375F37EC
:101A400000010101602B000111EF0DF08986010EEC
:101A50000101606F0001010160511908D8B003D085
:101A600000015FEF0DF00001D89001015C375D3798
:101A70005E375F37D8A003D0000143EF0DF00001BF
:101A8000899244EF0DF08982898489940101605123
:101A90000908D8A003D000015AEF0DF0000180B072
:101AA00055EF0DF0D89056EF0DF0D8800101633757
:101AB000643700010101602B00012BEF0DF08996C6
:101AC00001016351016E6451026E0001000C080EA9
:101AD000016E000004008B969496040001016837A3
:101AE0008298D8B09488D8A094989486000182A651
:101AF00077EF0DF0012E69EF0DF004008B969496B0
:101B00000000948804000400948682A685EF0DF0FE
:101B1000016A040082B801808B969496829894980A
:101B2000000C080E01016C6F000100C06DF194887B
:101B30000400948682A69AEF0DF082B8D88082A81D
:101B4000D8900136040094968B9601016C2F02D038
:101B500004D00001000197EF0DF0948804008298F2
:101B60006D51D8A4949800010000948682A6B6EF27
:101B70000DF004008B969496040082989498000CC3
:101B8000010E0101596F0001E76B948804009486EF
:101B900004008298949804008B969496A00E0101FC
:101BA000686F000167EC0DF00101686B000167ECE4
:101BB0000DF00101686B000167EC0DF094980000D6
:101BC000948682A6E1EF0DF0040000000000000002
:101BD0009488040094880400948604008298949861
:101BE00004008B969496A10E0101686F000167ECCA
:101BF0000DF001015A6B000101015A510608D8B0DD
:101C000003D0000118EF0EF00001D40E01015A2597
:101C1000E96EEA6AD8B0EA2A010E006E000191EC82
:101C20000DF00150EF6E01015A2B0001FCEF0DF099
:101C3000D43D25EF0EF0D53D25EF0EF0006A91EC76
:101C40000DF090EF0EF076EF0EF00101596B5A6B2C
:101C5000000101015A510B08D8B003D000016FEF09
:101C60000EF000015C0E01015A25E96E010EEA6ECC
:101C7000D8B0EA2A5A510A08D8A003D0000145EF8B
:101C80000EF00001000E46EF0EF0010E01016A6F2A
:101C900000016AC100F091EC0DF001C05BF15BC185
:101CA000EFFF070E01015A25016E036AD8B0032A1F
:101CB0000150D40FE96E000E0320EA6EEF505B5D19
:101CC000D8A403D000016AEF0EF00001010E01015B
:101CD000596F000101015A2B000129EF0EF0DB536F
:101CE000D8A476EF0EF00101596B00019498000022
:101CF000948682A679EF0EF0040000000000000038
:101D000094880400E72BE7516308D8A090EF0EF009
:101D100001015953D8B403D00001EAEF0DF00001DE
:101D200001015953D8A403D000019AEF0EF000012D
:101D3000D56BD46B01015953D8A403D00001A5EF92
:101D40000EF00001000EA6EF0EF0010E016E000C69
:101D500001011C6B000101011C5100017FEC01F02D
:101D600001011C2B00019EA8B3EF0EF0AD6E0D0E0D
:101D700001011C5DD8B403D00001ABEF0EF0090ED9
:101D80001D6F00012E0E9EA8C3EF0EF0AD6E010177
:101D90001D2F02D004D000010001C2EF0EF0010E91
:101DA000926E000181EC03F001015B6B000104EC19
:101DB0000DF002C01DF101C01CF101011C515408BD
:101DC000D8B403D0000109EF0FF0000101011D514B
:101DD0004108D8B403D0000109EF0FF00001010160
:101DE0001C6B000101011C5100018EEC01F001018E
:101DF0001C2B00019EA8FAEF0EF0AD6E050E01013E
:101E00001C5DD8B403D00001F2EF0EF0000121EF09
:101E10000FF001011C6B000101011C51000199EC44
:101E200001F001011C2B00019EA814EF0FF0AD6E14
:101E3000090E01011C5DD8B403D000010CEF0FF0B6
:101E4000000101011C6B000101011C510001A6EC05
:101E500001F001011C2B00019EA82CEF0FF0AD6ECC
:101E60000F0E01011C5DD8B403D0000124EF0FF068
:101E7000070E1D6F00012E0E9EA83CEF0FF0AD6EF9
:101E800001011D2F02D004D0000100013BEF0FF033
:101E9000070E756F0001A6EC07F00150800B000AD9
:101EA000D8A46DEF0FF001011C6B000101011C5162
:101EB000000199EC01F001011C2B00019EA85EEFCE
:101EC0000FF0AD6E090E01011C5DD8B403D0000106
:101ED00056EF0FF0000185EF0FF001011C6B0001C0
:101EE00001011C5100018EEC01F001011C2B0001CD
:101EF0009EA878EF0FF0AD6E050E01011C5DD8B401
:101F000003D0000170EF0FF0000101011C6B000114
:101F100001011C510001B6EC01F001011C2B000174
:101F20009EA890EF0FF0AD6E0F0E01011C5DD8B4AE
:101F300003D0000188EF0FF0070E1D6F00012E0E79
:101F40009EA8A0EF0FF0AD6E01011D2F02D004D0AE
:101F5000000100019FEF0FF00001C0EC0DF0E7530E
:101F6000D8A4CDEF0FF001011C6B000101011C5141
:101F7000000199EC01F001011C2B00019EA8BEEFAD
:101F80000FF0AD6E090E01011C5DD8B403D0000145
:101F9000B6EF0FF00001E5EF0FF001011C6B00013F
:101FA00001011C5100018EEC01F001011C2B00010C
:101FB0009EA8D8EF0FF0AD6E050E01011C5DD8B4E0
:101FC00003D00001D0EF0FF0000175EF3EF0FF0EDF
:101FD000956E816AF19E200E936E84808482848443
:101FE000969096929694F7EF0FF0E7EF0FF0020EAF
:101FF0000101686F0001C6EC01F08494020E01013A
:10200000686F0001C6EC01F01F0E0101756F000141
:10201000A6EC07F001C020F11F0E0101786F00014E
:1020200020C179F179EC07F0020E0101686F00011F
:10203000C6EC01F0070E0101756F0001A6EC07F078
:102040000150800B000AD8A442EF10F00101206B70
:10205000000101012051000102EC00F00101202BE0
:1020600000019EA831EF10F0AD6E0E0E0101205D53
:10207000D8B403D0000129EF10F0000E016E00016A
:1020800024EF11F00101786B210E796F000179ECDA
:1020900007F0020E0101686F0001C6EC01F00E0EA0
:1020A0000101786F480E796F000179EC07F00A0E94
:1020B0000101786F796B000179EC07F00B0E0101DB
:1020C000786F796B000179EC07F00C0E0101786FE5
:1020D000200E796F000179EC07F00D0E0101786F89
:1020E000020E796F000179EC07F0040E0101786FA0
:1020F000400E796F000179EC07F0010E0101786F55
:10210000460E796F000179EC07F0020E0101786F3D
:102110005F0E796F000179EC07F0030E0101786F13
:102120005E0E796F000179EC07F0070E0101786F00
:10213000FF0E796F000179EC07F00F0E0101786F47
:10214000796B000179EC07F00101786B610E796F12
:10215000000179EC07F0020E0101686F0001C6EC86
:1021600001F001011F6B000101011F510508D8B0EA
:1021700003D00001D5EF10F00001010E01011F2571
:10218000206F320E1F25E96EEA6AD8B0EA2A0001F4
:10219000EFCF21F120C178F121C179F179EC07F07D
:1021A00001011F2B0001B4EF10F001011F6B0001B2
:1021B00001011F510708D8B003D00001F3EF10F060
:1021C0000001080E01011F25206F000120C178F1D8
:1021D000FF0E0101796F000179EC07F001011F2B5F
:1021E0000001D8EF10F0070E0101786F470E796FEC
:1021F000000179EC07F0470E386E0101786B200E74
:10220000796F000179EC07F00C0E0101786F040E74
:10221000796F000179EC07F00D0E0101786F796B91
:10222000000179EC07F0070E0101786FFF0E796F5E
:10223000000179EC07F00101786B220E796F000143
:1022400079EC07F0010E016E000C016A026A006A67
:10225000036A01017651D8B403D0000137EF11F0C1
:102260007551D8A403D0000162EF11F00001100EE7
:102270000101776F0001D890010173377437003680
:1022800003367651035CD8B403D000014BEF11F054
:102290007551005C0001D8A057EF11F00101755194
:1022A000005ED8A003067651035ED8800001013697
:1022B00002360101772F02D004D0000100013BEF6C
:1022C00011F000010000000C01016A6B0001010126
:1022D0006A516A2B6B0FE96E010EEA6ED8B0EA2ADA
:1022E000000168C174F167C173F10101766B0A0ED8
:1022F000756F000125EC11F00050300FEF6E68C1D2
:1023000074F167C173F10101766B0A0E756F0001FC
:1023100025EC11F002C068F101C067F101016751BD
:102320006811D8B403D0000167EF11F000016AC151
:1023300069F101016A53D8A403D00001B3EF11F091
:10234000000101016A076B0E6A25E96E010EEA6E53
:10235000D8B0EA2A0001EFCF70F170C171F19FECA3
:1023600008F099EF11F001016951016E0001000CB4
:102370002986298429980101216B0001010121513D
:10238000000143EC01F00101212B00019EA8C6EFE2
:1023900011F0AD6E0D0E0101215DD8B403D0000126
:1023A000BEEF11F0686B00011CC067F164EC11F026
:1023B0002E0E0101716F00019FEC08F00101686BA6
:1023C00000011BC067F164EC11F02E0E0101716F6A
:1023D00000019FEC08F00101686B00011AC067F171
:1023E00064EC11F02E0E0101716F00019FEC08F0FA
:1023F0000101686B000119C067F164EC11F0000C79
:102400002986298429980101216B000101012151AC
:10241000000152EC01F00101212B00019EA80EEFFA
:1024200012F0AD6E0B0E0101215DD8B403D0000196
:1024300006EF12F0686B000124C067F164EC11F044
:102440002E0E0101716F00019FEC08F00101686B15
:10245000000123C067F164EC11F02E0E0101716FD1
:1024600000019FEC08F00101686B000122C067F1D8
:1024700064EC11F02E0E0101716F00019FEC08F069
:102480000101686B000121C067F164EC11F0000CE0
:102490002986298429980101216B0001010121511C
:1024A000000160EC01F00101212B00019EA856EF14
:1024B00012F0AD6E0E0E0101215DD8B403D0000103
:1024C0004EEF12F0686B000128C067F164EC11F068
:1024D0002E0E0101716F00019FEC08F00101686B85
:1024E000000127C067F164EC11F02E0E0101716F3D
:1024F00000019FEC08F00101686B000126C067F144
:1025000064EC11F02E0E0101716F00019FEC08F0D8
:102510000101686B000125C067F164EC11F0000C4B
:10252000010124AF03D00001AFEF12F00F0E006ED7
:10253000233900160A0E005CD8A003D00001A6EFD4
:1025400012F0300E00260001AAEF12F00101245112
:102550000026000100509EA8ABEF12F0AD6E0F0EEA
:10256000010123170A0E235DD8A003D00001BDEF9F
:1025700012F0300E0001C1EF12F00101249F24512E
:10258000000101012327235100019EA8C5EF12F08D
:10259000AD6E000C0101226B00010101225100010E
:1025A00070EC01F00101222B00019EA8D5EF12F082
:1025B000AD6E0C0E0101225DD8B403D00001CDEF49
:1025C00012F0216B0001010121510408D8B003D0A1
:1025D000000108EF13F00001320E01012125E96E20
:1025E000EA6AD8B0EA2A0001EFCF22F122C123F132
:1025F000370E0101246F000190EC12F03A0E9EA8F4
:10260000FFEF12F0AD6E0101212B0001E3EF12F09C
:1026100037C023F1370E0101246F000190EC12F056
:10262000200E9EA811EF13F0AD6E000C25C128F10D
:102630000101296B000124C103F0000E01012811E2
:10264000266F03502911276F2651016E2751026E04
:102650000001000C0101236B2151000B006E22517F
:10266000800B036E00500310D8A403D0000149EF83
:1026700013F0000101012353D8A403D0000145EF5A
:1026800013F00001000E46EF13F0010E0101236F5D
:10269000000101012151000B006E2251400B036E1D
:1026A00000500310D8A403D0000167EF13F000011D
:1026B00001012353D8A403D0000163EF13F00001FC
:1026C000000E64EF13F0010E0101236F0001010100
:1026D0002151000B006E2251100B036E00500310AD
:1026E000D8A403D0000185EF13F0000101012353AA
:1026F000D8A403D0000181EF13F00001000E82EF97
:1027000013F0010E0101236F000101012151080B9B
:10271000006E2251000B036E00500310D8A403D0AA
:102720000001A3EF13F0000101012353D8A403D04B
:1027300000019FEF13F00001000EA0EF13F0010E57
:102740000101236F0001010121512125246F225134
:102750002221256F23512425016E000E2521036EB1
:102760000350026E0001C7EF13F00101206B00015E
:10277000010120510708D8B003D00001D0EF13F0B9
:1027800000011FC122F11EC121F12AEF13F002C086
:102790001FF101C01EF10101202B0001B8EF13F061
:1027A00001011E51016E1F51026E000120EF18F051
:1027B000010125510408D8A003D00001F2EF13F065
:1027C0000001FF0AD8A4EEEF13F001012451DC0848
:1027D000D8A003D00001F2EF13F00001000E016E4B
:1027E00000EF14F021EC08F025C170F024C16FF067
:1027F00070C076F16FC075F185EC07F0010E016EC7
:10280000000C030E01012425E96E000E2521EA6E5D
:102810000001EFCF26F126C172F173EC08F0020E31
:1028200001012425E96E000E2521EA6E0001EFCF9B
:1028300026F126C172F173EC08F0010E0101242586
:10284000E96E000E2521EA6E0001EFCF26F126C1C8
:1028500072F173EC08F001012451E96E2551EA6E22
:102860000001EFCF26F126C172F173EC08F0000CE5
:10287000010122512207000AD8A403D0000149EF28
:1028800014F000010101726B000173EC08F038EFE5
:1028900014F065EF16F001012951036E2851D8B4E8
:1028A000290728070310D8A403D000016CEF14F007
:1028B000000101012751036E2651262BD8B4272B86
:1028C000E96E000103C0EAFFEFCF2AF12AC172F1DD
:1028D00073EC08F04BEF14F0000C25C126F126C173
:1028E00072F173EC08F024C172F173EC08F0000C83
:1028F000030E01012425E96E000E2521EA6E000178
:10290000EFCF26F126C173F14CEC08F0020E010165
:102910002425E96E000E2521EA6E0001EFCF26F195
:1029200026C173F14CEC08F0010E01012425E96E7B
:10293000000E2521EA6E0001EFCF26F126C173F1CA
:102940004CEC08F001012451E96E2551EA6E0001BA
:10295000EFCF26F126C173F14CEC08F0000C2B6A86
:102960002BC02AF02990450E0101726F000173EC13
:1029700008F00101726B000173EC08F0C2C025F190
:10298000C1C024F16DEC14F00101726B000173EC15
:1029900008F0C52BC5C072F173EC08F00101256B7E
:1029A000246B00016DEC14F0640E0101726F0001E4
:1029B00073EC08F0AEC072F173EC08F00101256B06
:1029C000190E246F000178EC14F00101256BB30E91
:1029D000246F000178EC14F02A500101246F241FA9
:1029E000000124C172F173EC08F02B500101246F37
:1029F000241F000124C172F173EC08F00101256B62
:102A0000190E246F000101EC14F00101256BB30EC7
:102A1000246F000101EC14F0000C26C127F1010124
:102A2000286B000127C173F14CEC08F025C173F14C
:102A30004CEC08F0000C2990C3C02AF0C4C02BF065
:102A4000B8C025F1B7C024F16DEC14F0BAC025F17F
:102A5000B9C024F16DEC14F0E9C025F1E8C024F10F
:102A60006DEC14F00101256B190E246F000178EC58
:102A700014F00101256BB30E246F000178EC14F003
:102A80000101736B00014CEC08F0110E0101736F32
:102A900000014CEC08F0E9C026F1E8C025F10DEC8E
:102AA00015F029AE58EF15F0FF0E2B6E2BC02AF053
:102AB0002A500101246F241F000124C172F173EC1C
:102AC00008F02B500101246F241F000124C172F172
:102AD00073EC08F00DEF16F06EC025F16DC024F117
:102AE00021EC08F0FF0E0101766FF20E756F000108
:102AF00085EC07F0716A0101276BA60E266F296B22
:102B0000060E286F00014BEC14F00101276B320E0A
:102B1000266F296B060E286F00014BEC14F0ADC038
:102B200026F126C172F173EC08F0ACC072F173ECBF
:102B300008F00E0E01012427000E25230001B3EC3E
:102B400007F001012553D8B403D00001B7EF15F009
:102B50000001010124513B08D8B003D00001B7EFB8
:102B600015F000010101256B3C0E246F0001050EDC
:102B70000101786F000124C179F179EC07F025C1DA
:102B800026F1060E0101786F000126C179F179EC7A
:102B900007F00101786B240E796F000179EC07F0E2
:102BA000000C21EC08F02AC0C3F02BC0C4F00101D6
:102BB000236B226B7052D8B403D00001E6EF15F0FE
:102BC00000016F501C08D8B0EEEF15F01C0E6F5CC2
:102BD0000101226F000E7058236F0001080E0101E1
:102BE00022250001E86F000E010123210001E96F99
:102BF000140EE825C16F000EE921C26F0101256B9B
:102C0000246B0001D8EC13F0080EAD6FAC6B110E05
:102C1000AE6FAFEC14F01BEF15F06CEC15F0000C80
:102C2000299629942988080EAD6FAC6B110EAE6FF2
:102C3000B86B440EB76FBA6B430EB96F0101256BC9
:102C40001C0E246F0001D8EC13F0010E0101726F0D
:102C5000000173EC08F0010E0101726F000173ECCA
:102C600008F0060E0101726F000173EC08F001011B
:102C7000726B000173EC08F00101256BFF0E246FED
:102C8000000101EC14F00101726B000173EC08F01B
:102C9000060E0101726F000173EC08F00101726B06
:102CA000000173EC08F00101726B000173EC08F095
:102CB0000101256B190E246F000101EC14F00C0EBC
:102CC0000101226F000138EF14F00101276B320E71
:102CD000266F296B060E286F00014BEC14F0705024
:102CE0000108D8A083EF16F0D8A47CEF16F06F503F
:102CF0000708D8A083EF16F00101726B000173EC96
:102D000008F06FEF16F0630E0101726F000173ECB3
:102D100008F0820E0101726F000173EC08F0530E8F
:102D20000101726F000173EC08F0630E0101726F14
:102D3000000173EC08F0350E0101726F000173ECB5
:102D400008F0010E0101726F000173EC08F001013F
:102D50001E510F0B226F000122C172F173EC08F0BB
:102D60003D0E0101726F000173EC08F0070E0101C6
:102D7000726F000173EC08F0010E0101726F000127
:102D800073EC08F00101276B320E266F296B060EDB
:102D9000286F00014BEC14F00C0E0101726F000162
:102DA00073EC08F02998036A360EE96E03C0EAFF57
:102DB000ECCF23F1ED52EFCF22F123C125F122C157
:102DC00024F116EC13F002C021F101C020F121C161
:102DD00068F120C167F164EC11F001C01FF129888E
:102DE000060E01011F25226F000122C172F173EC52
:102DF00008F0000E81BA010E000AD8A416EF17F0F1
:102E00000101226B000101012251000104EC01F0DB
:102E10000009D8B414EF17F00101222B726F0001E2
:102E200073EC08F003EF17F02AEF17F00101226BA3
:102E3000000101012251000110EC01F00009D8B499
:102E40002AEF17F00101222B726F000173EC08F0DA
:102E500019EF17F021C168F120C167F164EC11F09E
:102E600001011E510308D8B403D0000178EF17F018
:102E70000001360E0101726F000173EC08F0040EC0
:102E80000101726F000173EC08F0010E0101256F62
:102E9000090E246F000101EC14F0320E0101726F73
:102EA000000173EC08F0040E0101726F000173EC75
:102EB00008F00101256BFB0E246F000101EC14F0FA
:102EC000390E0101726F000173EC08F0020E01016E
:102ED000726F000173EC08F0050E0101726F0001C2
:102EE00073EC08F0DC0E0101726F000173EC08F066
:102EF000370E0101726F000173EC08F0030E01013F
:102F0000726F000173EC08F0010E0101726F000195
:102F100073EC08F0030E0101726F000173EC08F00E
:102F20000C0E0101726F000173EC08F0FF0E01013D
:102F3000726F000173EC08F001011E511308D8B440
:102F400003D00001BFEF17F00001EA6AA60EE96E98
:102F5000010EE26E030EE16E060E016EE6CFEEFF8D
:102F6000012EAEEF17F0040E016EEA6AB30EE96EA1
:102F7000FF0EEE6E012EB8EF17F0D3EF17F0060E2E
:102F8000016EEA6AA60EE96EFF0EEE6E012EC4EF28
:102F900017F0040E016EEA6AB30EE96EFF0EEE6ED4
:102FA000012ECEEF17F0D1EC15F0B4EF18F00101BF
:102FB000625164030001F3CF01F0F4CF00F001018E
:102FC0006503F350002663516403F3500020026E42
:102FD0000001000CEC53D8A442EF18F01C6A1B6AE5
:102FE0001A6A196A036A360EE96E03C0EAFFECCF6B
:102FF0001FF1ED52EFCF1EF11FC125F11EC124F1CB
:1030000016EC13F002C01DF101C01CF1F66BF56B5C
:103010000101256BED0E246F276B266B000136EC4A
:1030200007F00101256BEF0E246F276B266B000163
:1030300036EC07F01DC11FF11CC11EF1B5EF13F0F6
:1030400002C01FF101C01EF101011E511F0B006ED5
:103050001F51000B036E0050140F0001F16F000EA2
:103060000320F26FF2C0F4F0F1C0F3F01DC100F1E3
:103070001CC1FFF0F4C002F1F3C001F1010EEC6FCE
:10308000B4EF18F0EC2D47EF18F051EF18F0EC51B9
:103090000308D8B451EF18F0EC511308D8A4B4EFDA
:1030A00018F00101256BED0E246F0001F2C027F12D
:1030B000F1C026F136EC07F00152D8B4B4EF18F0A5
:1030C000EC2D65EF18F06AEF18F0EC510308D8A466
:1030D000A5EF18F0010E1626F2510408D8A07DEFD6
:1030E00018F0D8A479EF18F0F151AF08D8A07DEF0F
:1030F00018F0F351F127F451F22301011E6B000186
:1031000001011E510001F2EC00F001011E2B000133
:103110009EA888EF18F0AD6E120E01011E5DD8B4A6
:1031200003D0000180EF18F0060E1F6F00012E0E75
:103130009EA898EF18F0AD6E01011F2F02D004D0A9
:103140000001000197EF18F000012B6A2BC02AF054
:103150002A52D8A4AFEF18F02990B0EF18F02980C8
:10316000ECC01EF110EF16F0EC513008D8B4BEEFF1
:1031700018F0EC511308D8A401EF19F00101256BE8
:10318000EF0E246F276B140E266F000136EC07F04C
:103190000152D8B4FDEF18F0F52BD8B4F62BF95145
:1031A000F55DD8A4ECEF18F0FA51F65DD8A4ECEF79
:1031B00018F00101636B050E626F0001F4C065F148
:1031C000F3C064F1D7EC17F002C0F2F001C0F1F0E7
:1031D000130EEC6FFDEF18F0F851F65DD8A0FDEF7F
:1031E00018F0D8A4F9EF18F0F751F55DD8A0FDEF6D
:1031F00018F0FAC0F6F0F9C0F5F0010E016E03EF19
:1032000019F0000E016E18EF3FF00101246B256BE1
:10321000000101012551225DD8B003D0000147EF24
:1032200019F00001D8A41EEF19F001012151245D0D
:10323000D8A003D0000147EF19F00001010E0101F1
:103240006C6F230E6B6F000188EC0BF00152D8B449
:1032500047EF19F001011F512011D8A403D000013C
:1032600040EF19F0000101012051036E1F511F2B87
:10327000D8B4202BE96E000103C0EAFF23C1EFFFA1
:103280000101242BD8B4252B000109EF19F001010D
:103290002451016E2551026E0001000C01012051E4
:1032A0005E08D8A003D000015EEF19F00001E70E20
:1032B00001012025206F00016BEF19F00101205161
:1032C0004508D8B003D000016BEF19F00001190ECA
:1032D00001012027000101012051016E0001000CB5
:1032E0003D6A3C6A070E0101756F0001A6EC07F00C
:1032F0000150100B000AD8B485EF19F02E0E9EA8CD
:103300007FEF19F0AD6EF5EC0FF00101786B600EF8
:10331000796F000179EC07F0070E0101756F00016C
:10332000A6EC07F001011D6B000101C01CF10101B9
:10333000786B200E796F000179EC07F038500101AD
:103340001C5DD8B403D00001AFEF19F000010101FA
:103350001D53D8A403D000015FEF1AF0000138C05C
:1033600039F00101206B000138C01FF11FC13BF093
:103370003A6A6EEC09F0120E0101746F0001B6ECAE
:103380000AF00101206B9C0E1F6F226B120E216F41
:10339000000105EC19F0120E3A26000E3B226EECED
:1033A00009F09FC03DF09EC03CF09C51010B000A0B
:1033B000D8B401EF1AF03D52D8A4E4EF19F03C5014
:1033C0003F08D8B001EF1AF03D500508D8A001EF32
:1033D0001AF0D8A4F1EF19F03C50EE08D8A001EF94
:1033E0001AF0120E3C5E000E3D5AADC025F1ACC085
:1033F00024F116EC13F002C0ADF001C0ACF01BEFED
:103400001AF03D6A3C6A01011F6B000101011F5166
:10341000000112EC00F001011F2B00019EA80EEF2D
:103420001AF0AD6E0D0E01011F5DD8B403D000017E
:1034300006EF1AF000019D514508D8B029EF1AF0A7
:103440009D515E08D8A029EF1AF09DC038F04CEFCE
:103450001AF03D6A3C6A01011F6B000101011F5116
:10346000000121EC00F001011F2B00019EA836EFA6
:103470001AF0AD6E0D0E01011F5DD8B403D000012E
:103480002EEF1AF0010E38241F6F00011FC120F12A
:103490004EEC19F001C038F0010E385C01011F6FCD
:1034A00000011FC120F14EEC19F001C01EF1030E06
:1034B0000101786F00011EC179F179EC07F03C52EF
:1034C000D8A46AEF1AF03D52D8A46AEF1AF0000EA1
:1034D0006BEF1AF0010E016E4AEF3FF0716A6E6AEF
:1034E00071C06DF06EC070F06DC06FF02B6A2BC0B4
:1034F0002AF02A52D8A480EF1AF0299081EF1AF00E
:1035000029800101766B756B000185EC07F0000CDA
:10351000010E01016C6F5A0E6B6F000188EC0BF00D
:103520000152D8B4A1EF1AF001015A51595DD8B433
:1035300003D00001A1EF1AF00001010E016EA3EF0C
:103540001AF0000E016E000C010E01016C6F240ECA
:103550006B6F000188EC0BF00152D8B4DEEF1AF06B
:10356000010E01016C6F250E6B6F000188EC0BF0F2
:103570000152D8B4DEEF1AF00101296B000124C119
:1035800028F128C12BF101012A6B036A25512A1168
:10359000266F03502B11276F000123C103F0010197
:1035A0002251E96E000103C0EAFF27C1ECFFED5292
:1035B00026C1EFFF010E016EE0EF1AF0000E016E62
:1035C000000C040E0101236F030E2125256F000E50
:1035D0002221266F000126C16CF125C16BF188EC18
:1035E0000BF00152D8B42DEF1BF0020E0101212582
:1035F000266F000E2221276F000127C16CF126C122
:103600006BF188EC0BF00152D8B42DEF1BF0010EDA
:1036100001012125276F000E2221286F000128C1FA
:103620006CF127C16BF188EC0BF00152D8B42DEF8F
:103630001BF001012151286F2251296F000129C17E
:103640006CF128C16BF188EC0BF00152D8B42DEF6E
:103650001BF0010E016E2FEF1BF0000E016E000C2F
:10366000010122512311D8A403D000014DEF1BF01A
:103670000001010E01016C6F240E6B6F000188ECDC
:103680000BF00152D8B44DEF1BF001012251D8B418
:1036900023072207000130EF1BF001012253D8B4A9
:1036A00003D0000161EF1BF0000101012353D8B4E6
:1036B00003D0000161EF1BF00001010E016E63EF0A
:1036C0001BF0000E016E000C030E01011E25E96EB9
:1036D000000E1F21EA6E0001EFCF20F120C159F149
:1036E00088EC1AF00152D8B4AEEF1BF0020E0101C3
:1036F0001E25E96E000E1F21EA6E0001EFCF21F1B9
:1037000021C159F188EC1AF00152D8B4AEEF1BF088
:10371000010E01011E25E96E000E1F21EA6E000157
:10372000EFCF22F122C159F188EC1AF00152D8B43E
:10373000AEEF1BF001011E51E96E1F51EA6E000150
:10374000EFCF23F123C159F188EC1AF00152D8B41C
:10375000AEEF1BF0010E016EB0EF1BF0000E016E1C
:103760008BEF1CF00101216B00016EEC1AF00101DE
:103770001E2D02D004D000010001CAEF1BF0000191
:10378000060E016EEA6AA60EE96EFF0EEE6E012EBF
:10379000C5EF1BF00101256B010E246F00016DECDC
:1037A00014F0080E0101256F246B00016DEC14F07C
:1037B000060E0101726F000173EC08F0040E0101A6
:1037C000726F000173EC08F00101206B00011EC153
:1037D0001FF120C125F11FC124F16DEC14F001018E
:1037E000276B320E266F296B060E286F00014BECFB
:1037F00014F00101256B190E246F000101EC14F087
:103800000101276BA60E266F296B060E286F00019B
:103810004BEC14F00101256BB30E246F000101EC99
:1038200014F0080EAD6F060EAC6F6CEC15F0A6EF41
:103830001CF00101596B000188EC1AF00152D8B458
:10384000DFEF1CF0010E0101596F000188EC1AF046
:103850000152D8B4DFEF1CF0080E0101596F0001CE
:1038600088EC1AF00152D8B4DFEF1CF00101596B5B
:10387000000188EC1AF00152D8B4DFEF1CF0060EFC
:103880000101596F000188EC1AF00152D8B4DFEF42
:103890001CF0040E0101596F000188EC1AF001526E
:1038A000D8B4DFEF1CF0010E0101236F1C0E226F54
:1038B0000001A4EC1AF00152D8B4DFEF1CF00101B2
:1038C000206BBB0E1F6F226B060E216F000105ECF3
:1038D00019F001500210D8B4DFEF1CF00101226B87
:1038E000B30E216F0001E1EC1AF00152D8B4DFEF02
:1038F0001CF00101236B060E226F000130EC1BF05F
:103900000152D8B4DFEF1CF001011F6B190E1E6FBE
:10391000000164EF1BF00152D8B4DFEF1CF001018D
:103920001C2D02D004D000010001ACEF1CF00001FE
:1039300001011D53D8B403D00001ACEF1CF000010D
:10394000020E01011E6F0001B2EF1BF0010E016EAD
:10395000E1EF1CF0DFEF1CF001011C510208D8B4AC
:1039600003D00001DFEF1CF0000101011D53D8B4AA
:1039700003D00001DFEF1CF000012550B35DD8A497
:10398000DEEF1CF02650B45DD8A4DEEF1CF027500B
:10399000B55DD8A4DEEF1CF02850B65DD8A4DEEFEC
:1039A0001CF0EA6A2C0EE96EE26ABB0EE16E060EAE
:1039B000016EE6CFEEFF012ED9EF1CF0148C000E45
:1039C000016E5FEF3FF0010E01016C6F210E6B6F16
:1039D000000188EC0BF00152D8B4F3EF1CF0010E9B
:1039E000016EF5EF1CF0000E016E000C01011E517E
:1039F0003E24206F1F513F20216F3D5CD8B003D083
:103A0000000114EF1DF00001D8A410EF1DF03C5090
:103A10000101205DD8A003D0000114EF1DF00001CA
:103A200021C13DF020C13CF0415001011E25206F15
:103A3000000E1F21216F2153D8B403D000012DEFB8
:103A40001DF0000140500101205DD8A003D000010D
:103A50002DEF1DF0000120C140F0B6EF1DF02990C0
:103A6000299A2B6A2BC02AF0450E0101596F0001DB
:103A700088EC1AF00152D8B4BAEF1DF0E3EC1CF058
:103A80000152D8B4BAEF1DF00101236BC10E226FB1
:103A90000001A4EC1AF00152D8B4BAEF1DF00101F4
:103AA000236B020E226F000130EC1BF00152D8B4E0
:103AB000BAEF1DF00101236B020E226F000130EC02
:103AC0001BF00152D8B4BAEF1DF0E3EC1CF0015228
:103AD000D8B4BAEF1DF001016C6BAE0E6B6F000134
:103AE00088EC0BF00152D8B4BAEF1DF00101236B42
:103AF000020E226F000130EC1BF00152D8B4BAEF75
:103B00001DF00101226BB30E216F0001E1EC1AF0F0
:103B10000152D8B4BAEF1DF00101226BAF0E216F34
:103B20000001E1EC1AF00152D8B4BAEF1DF02A3CC2
:103B3000BAEF1DF02B3CBAEF1DF0C253D8A4A6EF8C
:103B40001DF0C1511408D8B0BAEF1DF0140EC15DBC
:103B500001011C6F000E0001C25901011D6F00011F
:103B60001DC11FF11CC11EF1F6EF1CF0010E016E0C
:103B7000BCEF1DF0000E016E6AEF3FF03D500101F9
:103B8000235DD8B003D00001D7EF1DF00001D8A409
:103B9000D3EF1DF0010122513C5CD8A003D00001FD
:103BA000D7EF1DF00001000E016EE6EF1DF023C1FE
:103BB00075F122C174F13AEC09F023C13FF022C142
:103BC0003EF0416A41C040F0010E016E000C01015F
:103BD000256B266B276B000121EC08F001016E6B51
:103BE0002A0E6F6F0001FAEC0AF00152D8A4FDEF23
:103BF0001DF04052D8B453EF1EF040C024F1010133
:103C000024512625286F000E2721296F2351295D75
:103C1000D8B003D0000126EF1EF00001D8A41AEF9F
:103C20001EF001012251285DD8B003D0000126EF1B
:103C30001EF00001010E0101256F2651225D006E6C
:103C400027512359036E0050246F0001416A01017E
:103C50002451415CD8A003D000013FEF1EF00001C9
:103C6000420E4124E96EEA6AD8B0EA2AEFCF28F181
:103C700028C172F173EC08F0412A27EF1EF0010110
:103C800024513E26000E3F2224512627000E2723D2
:103C90002553D8A403D0000151EF1EF0000153EFCB
:103CA0001EF0EEEF1DF06E50705CD8A065EF1EF0B8
:103CB000D8A460EF1EF06F506D5CD8B065EF1EF0B9
:103CC00070C003F06F5068EF1EF06EC003F06D50CF
:103CD0006D6E03C06EF001012651016E2751026E18
:103CE0000001000C29902B6A2BC02AF0140EC15D34
:103CF0000101226F000E0001C2590101236F040E61
:103D0000225D206F000E2359216F19500001AF5D15
:103D1000D8A4F9EF1EF01A50B05DD8A4F9EF1EF048
:103D20001B50B15DD8A4F9EF1EF01C50B25DD8A4B1
:103D3000F9EF1EF0080E0101596F000188EC1AF02E
:103D40000152D8B4F9EF1EF00101596B000188EC63
:103D50001AF00152D8B4F9EF1EF0010E0101236FE1
:103D60001C0E226F0001A4EC1AF00152D8B4F9EF36
:103D70001EF03FC01FF13EC01EF121C123F120C142
:103D800022F130EC1BF01FC123F11EC122F1BEEC69
:103D90001DF02A3CF9EF1EF02B3CF9EF1EF0AFECC2
:103DA00014F00101256B246B00016DEC14F0080E7A
:103DB00001011D271D510708D8B003D00001E7EF0E
:103DC0001EF0000101011C2BD8B41D2B00011DC1E8
:103DD00025F11CC124F16DEC14F021C123F120C1A7
:103DE00022F1E7EC1DF06CEC15F0010E016EFBEF1B
:103DF0001EF0000E016E73EF3FF03E503C5C006E13
:103E00003F503D58036E0050016E0350026EE7EFC5
:103E100021F001012353D8A403D0000136EF1FF095
:103E20000001010E01016C6F240E6B6F000188EC24
:103E30000BF00152D8B436EF1FF022C103F001019C
:103E40002151E96E000103C0EAFF01012451EF5C3A
:103E5000D8B403D0000136EF1FF000010101212B7F
:103E6000D8B4222B2307000109EF1FF001012353CF
:103E7000D8B403D0000142EF1FF00001010E016E23
:103E800044EF1FF0000E016E99EF1FF00101206B4F
:103E9000298A020E596F000188EC1AF00152D8B439
:103EA00074EF21F0E3EC1CF00152D8B474EF21F070
:103EB000060E0101596F000188EC1AF00152D8B4C6
:103EC00074EF21F00101236B0D0E226F000130EC25
:103ED0001BF00152D8B474EF21F0010E0101226FE2
:103EE000110E216F0001E1EC1AF00152D8B474EF09
:103EF00021F0010E0101226F150E216F0001E1EC8E
:103F00001AF00152D8B474EF21F00101236B040EB2
:103F1000226F000130EC1BF00152D8B474EF21F095
:103F20000101226B320E216F060E236F000109EF93
:103F30001FF00152D8B474EF21F00101236BCA0EB7
:103F4000226F000130EC1BF00152D8B474EF21F065
:103F5000299829942986630E0101596F000188EC84
:103F60001AF00152D8B474EF21F0820E0101596F9A
:103F7000000188EC1AF00152D8B474EF21F0530E0E
:103F80000101596F000188EC1AF00152D8B474EFA6
:103F900021F0630E0101596F000188EC1AF0015203
:103FA000D8B474EF21F0010E01016C6F1E0E6B6F1F
:103FB000000188EC0BF00152D8B4BBEF20F00101F6
:103FC0001E3D02D004D000010001EAEF1FF0000105
:103FD000BBEF20F0010E01016C6F1F0E6B6F000133
:103FE00088EC0BF00152D8B4BBEF20F001011E5158
:103FF0003508D8B403D0000112EF20F00001010110
:104000001F2D02D004D00001000112EF20F00001AA
:10401000010E01016C6F200E6B6F000188EC0BF03C
:10402000B9EF20F001011E513308D8B403D00001CC
:104030002EEF20F0000101011F510408D8B403D075
:1040400000012EEF20F00001010E0101226F0D0E84
:10405000216F0001E1EC1AF0B9EF20F001011E51CF
:104060003608D8B403D000016AEF20F00001010146
:104070001F510408D8B403D000016AEF20F00001FA
:1040800001011553D8B403D000016AEF20F00001FC
:1040900001011653D8B403D000016AEF20F00001EB
:1040A00001011753D8B403D000016AEF20F00001DA
:1040B00001011853D8B403D000016AEF20F00001C9
:1040C000010E0101226F150E216F0001E1EC1AF0C3
:1040D000B9EF20F001011E2D02D004D00001000133
:1040E0008EEF20F0000101011F510408D8B403D065
:1040F00000018EEF20F00001010120510508D8B425
:1041000003D000018EEF20F000010101226B210E8F
:10411000216F0001E1EC1AF0B9EF20F001011E510E
:104120000308D8B403D00001B2EF20F00001010170
:104130001F510308D8A003D00001B2EF20F0000106
:10414000010120510508D8B403D00001B2EF20F0DE
:1041500000010101226B250E216F0001E1EC1AF034
:10416000B9EF20F00101236B00011FC122F130ECF7
:104170001BF0D3EF1FF0EC2DEDEF20F001012051EB
:104180000208D8B403D00001EDEF20F00001010EC9
:10419000EA6E030EE96EE26AA60EE16E060E016E8D
:1041A000E6CFEEFF012ED0EF20F018C10CF117C1C1
:1041B0000BF116C10AF115C109F114C1FEF013C1CA
:1041C000FDF012C1FCF011C1FBF0F4C0F2F0F3C03D
:1041D000F1F0030EEC6F74EF21F0EC510308D8B44A
:1041E000F7EF20F0EC511308D8A460EF21F00101A3
:1041F00020510508D8B403D0000160EF21F0000180
:10420000A80EF86FC00EF76F01011053D8B403D099
:1042100000012DEF21F0000101010F53D8B403D0AC
:1042200000012DEF21F0000101010E51A808D8B0C6
:1042300003D000012DEF21F00001D8A429EF21F0D7
:1042400001010D51BF08D8B003D000012DEF21F0BE
:1042500000010EC1F8F00DC1F7F0F853D8A439EF02
:1042600021F0F7513B08D8A039EF21F0F86B3C0E54
:10427000F76FD890F831FA6FF731F96FF66BF56B8D
:10428000FEC01CF0FDC01BF0FCC01AF0FBC019F012
:10429000B8EC11F000EC12F048EC12F0CAEC12F09D
:1042A000166A0D0E9EA852EF21F0AD6E0A0E9EA862
:1042B00057EF21F0AD6E300EEC6F148E74EF21F0DD
:1042C000EC510308D8B46AEF21F0EC511308D8A4DC
:1042D00074EF21F0010120510608D8B403D0000189
:1042E00074EF21F00001EC6B6BEF22F02B6A2BC016
:1042F0002AF0299E29900101236BB90E226F00013B
:10430000A4EC1AF00152D8B46FEF22F00101236B34
:10431000B70E226F0001A4EC1AF00152D8B46FEF6F
:1043200022F00101236BE80E226F0001A4EC1AF0C9
:104330000152D8B46FEF22F00101236BEA0E226F15
:104340000001A4EC1AF00152D8B46FEF22F0E95347
:10435000D8A4B0EF21F0E8510708D8B06FEF22F0F1
:10436000E9510508D8A06FEF22F0D8A4BDEF21F0E5
:10437000E851C008D8A06FEF22F0EA51EB11D8B491
:10438000F7EF21F0E9C026F1E8C025F10DEC15F0BA
:104390000101256BAF0E246F000178EC14F00101D0
:1043A000256BB30E246F000178EC14F00101736BE0
:1043B00000014CEC08F0110E0101736F00014CEC90
:1043C00008F03FC01DF13EC01CF1FDEF1EF002C021
:1043D0001FF101C01EF11FC123F11EC122F130ECFB
:1043E0001BF01DC123F11CC122F1BEEC1DF0EA53EC
:1043F000D8A4FFEF21F0EB53D8B405EF22F02A3C0C
:104400006FEF22F02B3C6FEF22F00101216B0001D6
:104410006EEC1AF02B6A2BC02AF02990B7510708CE
:10442000D8A432EF22F0B853D8A432EF22F0010121
:10443000256B1C0E246F0001D8EC13F0080EE85D0C
:1044400001011E6F000E0001E95901011F6F0001FB
:104450001FC123F11EC122F1E7EC1DF0D1EC15F0D4
:104460006BEF22F0B7510D08D8A460EF22F0B853DB
:10447000D8A460EF22F02996299429880101256BA0
:104480001C0E246F0001D8EC13F001011E6B00011B
:1044900001011E51000130EC00F001011E2B716F73
:1044A00000019FEC08F00C0E01011E5DD8B403D092
:1044B000000148EF22F00001D1EC15F06BEF22F083
:1044C000B7514408D8A46BEF22F0B853D8A46BEFCF
:1044D00022F046EF1FF0010E016E71EF22F0000E88
:1044E000016E7CEF3FF001012351E96E2451EA6E29
:1044F0002551EF24016E2651EC20036EE906015090
:10450000EF6E000103C0ECFFE90601012351E96EE3
:104510002451EA6E0001ECCF28F1ED52EFCF27F1E4
:1045200001012851265DD8B003D00001B5EF22F07B
:104530000001D8A4A5EF22F001012551275DD8A0E4
:1045400003D00001B5EF22F00001020E0101232586
:10455000E96E000E2421EA6E010EEE26D8B003D0DB
:104560000001B5EF22F0EF2A0001000C948804004E
:10457000948604008298949804008B969496A00EDA
:104580000101686F000167EC0DF0D7C059F101011E
:104590005A6B000159C168F167EC0DF0D6C068F1A3
:1045A00067EC0DF094980000948682A6D5EF22F077
:1045B00004000000000000009488040094880400B7
:1045C000948604008298949804008B969496A10E89
:1045D0000101686F000167EC0DF0F2EF28F0D89050
:1045E000010159355A6FB40E5B6F000E926E8996B9
:1045F000010E5C6F000101015C512008D8B003D0AE
:1046000000010CEF23F00001898289948984010163
:104610005C2B0001FBEF22F0010E01015C6F000139
:1046200001015C512F08D8B003D000015CEF23F0EA
:10463000000101015C510F08D8B003D0000130EF38
:1046400023F00001D89001015A375B37D8A003D07E
:1046500000012FEF23F00001899230EF23F08982CF
:10466000899401015C510F08D8A003D0000147EFE5
:1046700023F0000180B240EF23F0D89041EF23F007
:10468000D88001015F376037613762370001898464
:1046900001015C510F08D8B403D0000157EF23F09B
:1046A0000001020E926E89948984899489840101A3
:1046B0005C2B000110EF23F05FC100F060C101F03E
:1046C00061C102F062C103F03FEF29F001015A6BB2
:1046D0005B6B5C6B5D6B5E6B5F6B606B616B626B8E
:1046E000636B646B656B666B676B686B696B6A6B3E
:1046F0005A6B000101015A510408D8B003D00001DF
:10470000A6EF23F00001010E01016C6F590E6B6FD3
:10471000000188EC0BF00152D8B4A6EF23F00101A0
:1047200059512008D8A003D00001A6EF23F00001C2
:10473000010159513D08D8A403D00001A6EF23F090
:10474000000101015A2B00017AEF23F001015A6B9D
:10475000000101015A510708D8B003D00001F8EF59
:1047600023F00001010E01016C6F590E6B6F000107
:1047700088EC0BF00152D8B4F8EF23F00101595145
:104780002008D8A003D00001F8EF23F000010101B8
:1047900059512608D8A403D00001F8EF23F00001F6
:1047A0005B0E01015A25E96E010EEA6ED8B0EA2AC5
:1047B00059516008D8A003D00001EFEF23F00001A9
:1047C000010159517A08D8B003D00001EFEF23F06E
:1047D000000101015951DF0B0001F2EF23F001014B
:1047E00059510001EF6E01015A2B0001A9EF23F08E
:1047F00001015A6B000101015A510408D8B003D0DD
:10480000000127EF24F00001010E01016C6F590E29
:104810006B6F000188EC0BF00152D8B427EF24F045
:10482000010159512008D8A003D0000127EF24F03E
:104830000001010159513D08D8A403D0000127EF20
:1048400024F0000101015A2B0001FBEF23F00101CC
:104850005A6B000101015A510708D8B003D000017A
:1048600079EF24F00001010E01016C6F590E6B6F9E
:10487000000188EC0BF00152D8B479EF24F001016B
:1048800059512008D8A003D0000179EF24F000018D
:10489000010159512608D8A403D0000179EF24F072
:1048A0000001630E01015A25E96E010EEA6ED8B0CF
:1048B000EA2A59516008D8A003D0000170EF24F013
:1048C0000001010159517A08D8B003D0000170EFFE
:1048D00024F0000101015951DF0B000173EF24F0B6
:1048E000010159510001EF6E01015A2B00012AEF1D
:1048F00024F001015A6B000101015A510708D8B098
:1049000003D00001A9EF24F000015B0E01015A253C
:10491000E96E010EEA6ED8B0EA2A0001EFCF6BF122
:10492000630E01015A25E96E010EEA6ED8B0EA2A3B
:10493000EF506B5DD8A403D00001A4EF24F0000178
:10494000000E016EFCEF24F001015A2B00017CEFF8
:1049500024F001015A6B000101015A510708D8B037
:1049600003D00001FAEF24F000010A0E01015A25DC
:104970006B6F00016BC1A9FFA86AA69CA69EA684C6
:10498000F250006EF29E0F01550EA76EAA0EA76E92
:10499000A6820001A6B2CAEF24F0A6940050F2123B
:1049A0000A0E01015A256B6F5B0E5A25E96E010E46
:1049B000EA6ED8B0EA2A0001EFCF6CF16BC1A9FF13
:1049C0006CC1A8FFA69CA69EA684F250006EF29E23
:1049D0000F01550EA76EAA0EA76EA6820001A6B201
:1049E000EFEF24F0A6940050F21201015A2B0001BF
:1049F000ACEF24F0010E016E89EF2BF001015A6B30
:104A00005B6B5C6B5D6B5E6B5F6B606B616B626B5A
:104A10005A6B000101015A510408D8B003D00001BB
:104A200036EF25F00001010E01016C6F590E6B6F1E
:104A3000000188EC0BF00152D8B436EF25F00101EB
:104A400059512008D8A003D0000136EF25F000010D
:104A5000010159513D08D8A403D0000136EF25F0DB
:104A6000000101015A2B00010AEF25F001015A6BE8
:104A7000000101015A510708D8B003D0000188EFA6
:104A800025F00001010E01016C6F590E6B6F0001E2
:104A900088EC0BF00152D8B488EF25F00101595190
:104AA0002008D8A003D0000188EF25F00001010103
:104AB00059513D08D8A403D0000188EF25F000012A
:104AC0005B0E01015A25E96E010EEA6ED8B0EA2AA2
:104AD00059516008D8A003D000017FEF25F00001F4
:104AE000010159517A08D8B003D000017FEF25F0B9
:104AF000000101015951DF0B000182EF25F0010196
:104B000059510001EF6E01015A2B000139EF25F0D8
:104B100001015B513008D8B403D00001D4EF25F077
:104B2000000101015C513508D8B403D00001D4EF75
:104B300025F0000101015D513408D8B403D0000113
:104B4000D4EF25F0000101015E513008D8B403D044
:104B50000001D4EF25F0000101015F513808D8B4FD
:104B600003D00001D4EF25F00001010160513608A7
:104B7000D8B403D00001D4EF25F000010101615148
:104B80003508D8B403D00001D4EF25F000010101AD
:104B900062513208D8B403D00001D4EF25F00001EF
:104BA000010E016E2CEF26F001015A6B000101018C
:104BB0005A510708D8B003D000012AEF26F00001AF
:104BC0005B0E01015A25E96E010EEA6ED8B0EA2AA1
:104BD000EF502008D8B403D0000103EF26F0000105
:104BE0000A0E01015A25646F000164C1A9FFA69C49
:104BF000A69EA680A850000AD8A403EF26F0010EB6
:104C0000016E2CEF26F05B0E01015A25E96E010EB4
:104C1000EA6ED8B0EA2A0001EFCF63F10A0E010173
:104C20005A25646F000164C1A9FFA69CA69EA680B8
:104C3000A8500101635DD8A403D0000125EF26F040
:104C40000001000E016E2CEF26F001015A2B00012D
:104C5000D7EF25F0010E016ECBEF2BF001015C6B5D
:104C60005D6B5E6B5F6B606B616B5F6B5E6B0001BE
:104C700001015F53D8B403D000016EEF26F00001AC
:104C800001015E510408D8B003D000016EEF26F098
:104C90000001010E01016C6F5B0E6B6F000188EC6F
:104CA0000BF00152D8B46EEF26F001015B512008E1
:104CB000D8A003D000016EEF26F0000101015B5186
:104CC0003D08D8A403D000016EEF26F000010101D9
:104CD0005E2BD8B45F2B000138EF26F001015F6B2B
:104CE0005E6B000101015F53D8B403D00001D7EF20
:104CF00026F0000101015E510408D8B003D0000184
:104D0000D7EF26F00001010E01016C6F5B0E6B6F97
:104D1000000188EC0BF00152D8B4D7EF26F0010166
:104D20005B512008D8A003D00001D7EF26F0000186
:104D300001015B512608D8A403D00001D7EF26F06B
:104D4000000101015B512F08D8A003D00001D0EF72
:104D500026F0000101015B513908D8B003D00001F1
:104D6000D0EF26F00001300E01015B5D606F616BDA
:104D700000015DC163F15CC162F10101656B0A0E66
:104D8000646F0001D7EC17F002C063F101C062F15B
:104D90000101605162255C6F615163215D6F00010B
:104DA00001015E2BD8B45F2B000172EF26F00101E8
:104DB0005C51016E5D51026E0001000C0F0E01018D
:104DC0005C175C510908D8B003D00001F4EF26F05D
:104DD0000001300E01015C255D6F00015DC171F1C4
:104DE0009FEC08F0FDEF26F0370E01015C255D6FAA
:104DF00000015DC171F19FEC08F0000C01015A390E
:104E00005B6F0F0E5B1700015BC15CF1DEEC26F0FF
:104E10005AC15CF1DEEC26F0000C59C1A9FFA69C3A
:104E2000A69EA680A8500008D8B02CEF27F059C144
:104E3000A9FFA69CA69EA680A8500408D8A02CEF87
:104E400027F059C1A9FFA69CA69EA680A850030FD3
:104E500001015B6F5C6B000159C1A9FFA69CA69E76
:104E6000A680A8500408D8B04BEF27F059C1A9FF7D
:104E7000A69CA69EA680A8500608D8A04BEF27F0B7
:104E800059C1A9FFA69CA69EA680A850FC0F0101AF
:104E90005B6F5C6B000159C1A9FFA69CA69EA68012
:104EA000A8500708D8A460EF27F059C1A9FFA69C15
:104EB000A69EA680A850010F01015B6F5C6B0001EC
:104EC00059C1A9FFA69CA69EA680A8500808D8A4F0
:104ED00075EF27F059C1A9FFA69CA69EA680A850F1
:104EE000FB0F01015B6F5C6B000101015B51016E07
:104EF0005C51026E0001000C59C1A9FFA69CA69E40
:104F0000A680A8500108D8B490EF27F059C1A9FF96
:104F1000A69CA69EA680A8500808D8A496EF27F0C5
:104F2000290E016E000E026EE4EF27F059C1A9FFB1
:104F3000A69CA69EA680A8500208D8B4AAEF27F087
:104F400059C1A9FFA69CA69EA680A8500308D8A474
:104F5000B0EF27F02A0E016E000E026EE4EF27F08C
:104F600059C1A9FFA69CA69EA680A8500408D8B443
:104F7000C4EF27F059C1A9FFA69CA69EA680A85001
:104F80000708D8A4CAEF27F02B0E016E000E026EA0
:104F9000E4EF27F059C1A9FFA69CA69EA680A850C1
:104FA0000508D8B4DEEF27F059C1A9FFA69CA69E3C
:104FB000A680A8500608D8A4E4EF27F0280E016EBA
:104FC000000E026EE4EF27F0000C006A91EC0DF089
:104FD00094980000948682A6EBEF27F0040000006E
:104FE000000000009488040092EF39F0010E0101E6
:104FF000396F010E3A6F010E3B6F3C6B010E3D6F36
:10500000010E3E6F010E3F6F010E406F010E416FAA
:10501000426B010E436F010E446F456B010E466FEC
:10502000010E476F486B010E496F010E4A6F4B6BC3
:10503000010E4C6F010E4D6F4E6B010E4F6F010E46
:10504000506F516B010E526F010E536F546B010E76
:10505000556F010E566F576B010E586F2B6A00018A
:105060002BC02AF02A52D8A439EF28F029903AEF21
:1050700028F02980298A470E0101596F000188EC28
:105080001AF00152D8B496EF39F0450E0101596F6C
:10509000000188EC1AF00152D8B496EF39F0540EA2
:1050A0000101596F000188EC1AF00152D8B496EF53
:1050B00039F0200E0101596F000188EC1AF02F0E13
:1050C0000101596F000188EC1AF00101216B000108
:1050D000010121510B08D8B003D00001A4EF28F042
:1050E0000001010E01016C6F250E6B6F000188EC51
:1050F0000BF00152D8B4A4EF28F00101255120088B
:10510000D8A003D00001A4EF28F00001010125512F
:105110003F08D8A403D00001A4EF28F00001070E37
:1051200001012125016E036AD8B0032A0150D40F72
:10513000E96E000E0320EA6E000125C1EFFF0101B8
:10514000212B000168EF28F0010121510B08D8B094
:1051500003D00001C1EF28F00001070E0101212555
:10516000016E036AD8B0032A0150D40FE96E000E15
:105170000320EA6EEF6A00010101212B0001A4EF78
:1051800028F0C0EC0DF00152D8B4C9EF28F0CCEFF4
:1051900028F0DB6BC0EC0DF02B6A2BC02AF02990B5
:1051A000706A280E6F6EE753D8A4F0EF28F0010163
:1051B000596B00010101595100014FEC00F0010150
:1051C000592B716F00019FEC08F01F0E0101595D12
:1051D000D8B403D00001DAEF28F0000192EF39F0E3
:1051E000B6EF22F0D451D511D8B490EF39F0010EBA
:1051F000006E91EC0DF001C023F1D451D8B4D50765
:10520000D407DA51010B000AD8B48AEF39F0010152
:1052100023514008D8B403D000018AEF39F00001CF
:10522000D451D511D8B48AEF39F0010E006E91EC4B
:105230000DF001C023F1D451D8B4D507D407300EF6
:105240000101235D246F23514008D8A003D0000141
:1052500030EF29F00001370E0101235D246F0001BA
:105260000101242D02D004D0000100011FEF2BF01A
:105270000001010E0101596F0001EFEF22F003C0A0
:1052800030F102C02FF101C02EF100C02DF101015B
:10529000216B0001010121511F08D8B003D000018A
:1052A00098EF29F0000130C134F12FC133F12EC144
:1052B00032F12DC131F1390E01012125E96E010EC6
:1052C000EA6ED8B0EA2A000134C15FF133C15EF161
:1052D00032C15DF131C15CF1010121515B6FD8A494
:1052E00003D0000183EF29F00001D89001015F3362
:1052F0005E335D335C335B2F02D004D000010001CC
:1053000075EF29F0000101015C51010B006E5D5148
:10531000000B016E5E51000B026E5F51000B036EBD
:10532000000100C0EFFF0101212B00014AEF29F02D
:10533000030E0101216F0001010121510608D8B0BF
:1053400003D000011DEF2AF0000101012151040DDD
:10535000F350390FE96E010EEA6ED8B0EA2AEF5227
:10536000D8A403D00001B9EF29F00001310EBAEF43
:1053700029F0300E01015B6F00015BC172F173EC2B
:1053800008F001012151040DF350010F390FE96EAE
:10539000010EEA6ED8B0EA2AEF52D8A403D0000179
:1053A000D6EF29F00001310ED7EF29F0300E0101C0
:1053B0005B6F00015BC172F173EC08F001012151D8
:1053C000040DF350020F390FE96E010EEA6ED8B0EA
:1053D000EA2AEF52D8A403D00001F3EF29F000012C
:1053E000310EF4EF29F0300E01015B6F00015BC15B
:1053F00072F173EC08F001012151040DF350030F19
:10540000390FE96E010EEA6ED8B0EA2AEF52D8A43D
:1054100003D0000110EF2AF00001310E11EF2AF045
:10542000300E01015B6F00015BC172F173EC08F09B
:105430000101212B00019CEF29F0000E81BA010E21
:10544000000AD8A4A8EF2AF00101216B0001010194
:1054500021510108D8B003D00001A8EF2AF00001C3
:1054600001012151040DF350390FE96E010EEA6E6E
:10547000D8B0EA2AEF52D8A403D0000144EF2AF0B2
:105480000001310E45EF2AF0300E01015B6F000183
:105490005BC172F173EC08F001012151040DF3506E
:1054A000010F390FE96E010EEA6ED8B0EA2AEF5209
:1054B000D8A403D0000161EF2AF00001310E62EFA1
:1054C0002AF0300E01015B6F00015BC172F173ECD9
:1054D00008F001012151040DF350020F390FE96E5C
:1054E000010EEA6ED8B0EA2AEF52D8A403D0000128
:1054F0007EEF2AF00001310E7FEF2AF0300E01011D
:105500005B6F00015BC172F173EC08F00101215186
:10551000040DF350030F390FE96E010EEA6ED8B097
:10552000EA2AEF52D8A403D000019BEF2AF0000131
:10553000310E9CEF2AF0300E01015B6F00015BC160
:1055400072F173EC08F00101212B000127EF2AF022
:10555000070E0101216F2151040DF350390FE96E3F
:10556000010EEA6ED8B0EA2AEF52D8A403D00001A7
:10557000BEEF2AF00001310EBFEF2AF0300E01011C
:105580005B6F00015BC172F173EC08F00101215106
:10559000040DF350010F390FE96E010EEA6ED8B019
:1055A000EA2AEF52D8A403D00001DBEF2AF0000171
:1055B000310EDCEF2AF0300E01015B6F00015BC1A0
:1055C00072F173EC08F001012151040DF350020F48
:1055D000390FE96E010EEA6ED8B0EA2AEF52D8A46C
:1055E00003D00001F8EF2AF00001310EF9EF2AF0A4
:1055F000300E01015B6F00015BC172F173EC08F0CA
:1056000001012151040DF350030F390FE96E010E12
:10561000EA6ED8B0EA2AEF52D8A403D0000115EF01
:105620002BF00001310E16EF2BF0300E01015B6FF5
:1056300000015BC172F173EC08F088EF39F00101F1
:1056400024510208D8B403D0000148EF2BF0000128
:10565000080EA96EA69CA69EA680A850000AD8A4F3
:1056600046EF2BF00101596B000101015951000176
:1056700067EC00F00009D8B446EF2BF00101592B7C
:10568000726F000173EC08F035EF2BF088EF39F002
:10569000010124510308D8B403D0000171EF2BF0AD
:1056A0000001080EA96EA69CA69EA680A85001081F
:1056B000D8A46FEF2BF00101596B00010101595182
:1056C000000167EC00F00009D8B46FEF2BF0010186
:1056D000592B726F000173EC08F05EEF2BF088EF2E
:1056E00039F0010124510408D8B403D000017EEF41
:1056F0002BF00001010E156E88EF39F001012451E5
:105700000608D8B403D00001C0EF2BF0000166EF0B
:1057100023F001C021F10101212D02D004D00001AC
:105720000001AAEF2BF000010101596B00010101FA
:105730005951000173EC00F00009D8B4A8EF2BF028
:105740000101592B726F000173EC08F097EF2BF0F9
:10575000BEEF2BF00101596B00010101595100010D
:1057600082EC00F00009D8B4BEEF2BF00101592BF8
:10577000726F000173EC08F0ADEF2BF088EF39F099
:10578000010124510708D8B403D00001E2EF2BF047
:105790000001FEEF24F001C021F101012153D8A442
:1057A00003D00001D8EF2BF00001310ED9EF2BF020
:1057B000300E0101596F000159C172F173EC08F00C
:1057C00088EF39F0010124510808D8B403D0000152
:1057D00049EF2CF000010101686B00011CC067F16A
:1057E00064EC11F02E0E0101726F000173EC08F0F1
:1057F0000101686B00011BC067F164EC11F02E0E13
:105800000101726F000173EC08F00101686B000187
:105810001AC067F164EC11F02E0E0101726F0001E5
:1058200073EC08F00101686B000119C067F164ECCA
:1058300011F01752D8A433EF2CF00101596B00017D
:105840000101595100018FEC00F00009D8B431EF8B
:105850002CF00101592B726F000173EC08F020EF5E
:105860002CF047EF2CF00101596B00010101595157
:1058700000019BEC00F00009D8B447EF2CF00101C7
:10588000592B726F000173EC08F036EF2CF088EFA3
:1058900039F0010124510908D8B403D00001F8EF10
:1058A0002DF00001A96A36C0A8FFA69CA69EA6847A
:1058B000F250006EF29E0F01550EA76EAA0EA76E53
:1058C000A6820001A6B262EF2CF0A6940050F2125C
:1058D000010EA96E37C0A8FFA69CA69EA684F25012
:1058E000006EF29E0F01550EA76EAA0EA76EA6823D
:1058F0000001A6B279EF2CF0A6940050F2122EEC23
:1059000026F002C05AF101C059F1020EA96E59C128
:10591000A8FFA69CA69EA684F250006EF29E0F01E0
:10592000550EA76EAA0EA76EA6820001A6B296EF2C
:105930002CF0A6940050F2122EEC26F002C05AF180
:1059400001C059F1030EA96E59C1A8FFA69CA69EDD
:10595000A684F250006EF29E0F01550EA76EAA0E9D
:10596000A76EA6820001A6B2B3EF2CF0A694005059
:10597000F2122EEC26F002C05AF101C059F1040EC9
:10598000A96E59C1A8FFA69CA69EA684F250006EDF
:10599000F29E0F01550EA76EAA0EA76EA6820001F9
:1059A000A6B2D0EF2CF0A6940050F2122EEC26F006
:1059B00002C05AF101C059F1050EA96E59C1A8FFE4
:1059C000A69CA69EA684F250006EF29E0F01550E74
:1059D000A76EAA0EA76EA6820001A6B2EDEF2CF06C
:1059E000A6940050F2122EEC26F002C05AF101C02B
:1059F00059F1130EA96E59C1A8FFA69CA69EA684B4
:105A0000F250006EF29E0F01550EA76EAA0EA76E01
:105A1000A6820001A6B20AEF2DF0A6940050F21261
:105A20002EEC26F002C05AF101C059F1140EA96EF5
:105A300059C1A8FFA69CA69EA684F250006EF29EB5
:105A40000F01550EA76EAA0EA76EA6820001A6B280
:105A500027EF2DF0A6940050F2122EEC26F002C093
:105A60005AF101C059F1150EA96E59C1A8FFA69CA3
:105A7000A69EA684F250006EF29E0F01550EA76EF0
:105A8000AA0EA76EA6820001A6B244EF2DF0A6943E
:105A90000050F2122EEC26F002C05AF101C059F16A
:105AA000160EA96E59C1A8FFA69CA69EA684F25008
:105AB000006EF29E0F01550EA76EAA0EA76EA6826B
:105AC0000001A6B261EF2DF0A6940050F2122EEC68
:105AD00026F002C05AF101C059F1170EA96E59C142
:105AE000A8FFA69CA69EA684F250006EF29E0F010F
:105AF000550EA76EAA0EA76EA6820001A6B27EEF73
:105B00002DF0A6940050F2122EEC26F002C05AF1AD
:105B100001C059F1180EA96E59C1A8FFA69CA69EF6
:105B2000A684F250006EF29E0F01550EA76EAA0ECB
:105B3000A76EA6820001A6B29BEF2DF0A69400509E
:105B4000F2122EEC26F002C05AF101C059F1190EE2
:105B5000A96E59C1A8FFA69CA69EA684F250006E0D
:105B6000F29E0F01550EA76EAA0EA76EA682000127
:105B7000A6B2B8EF2DF0A6940050F2122EEC26F04B
:105B800002C05AF101C059F11A0EA96E59C1A8FFFD
:105B9000A69CA69EA684F250006EF29E0F01550EA2
:105BA000A76EAA0EA76EA6820001A6B2D5EF2DF0B1
:105BB000A6940050F21203EC02F001C059F1060E57
:105BC000A96E59C1A8FFA69CA69EA684F250006E9D
:105BD000F29E0F01550EA76EAA0EA76EA6820001B7
:105BE000A6B2F0EF2DF0A6940050F21288EF39F033
:105BF000010124510A08D8B403D0000184EF2FF02A
:105C00000001010E926E81EC03F0040E0101226F7F
:105C10000001010122510708D8B003D00001C0EFF4
:105C20002EF0000122C15BF104EC0DF00101306B9C
:105C30002F6B000102C02EF101C02DF10101216B7B
:105C40000001010121511F08D8B003D000016FEFFE
:105C50002EF0000130C134F12FC133F12EC132F1E9
:105C60002DC131F1390E01012125E96E010EEA6ED7
:105C7000D8B0EA2A000134C15FF133C15EF132C10C
:105C80005DF131C15CF1010121515B6FD8A403D0FA
:105C900000015AEF2EF00001D89001015F335E330E
:105CA0005D335C335B2F02D004D0000100014CEF68
:105CB0002EF0000101015C51010B006E5D51000BE3
:105CC000016E5E51000B026E5F51000B036E00010E
:105CD00000C0EFFF0101212B000121EF2EF0010197
:105CE0003A53D8A403D000017AEF2EF00001310E10
:105CF0007BEF2EF0300E0101596F000159C172F196
:105D000073EC08F001013B53D8A403D000018DEFE0
:105D10002EF00001310E8EEF2EF0300E0101596F82
:105D2000000159C172F173EC08F001013C53D8A491
:105D300003D00001A0EF2EF00001310EA1EF2EF0F4
:105D4000300E0101596F000159C172F173EC08F076
:105D500001014153D8A403D00001B3EF2EF000019C
:105D6000310EB4EF2EF0300E0101596F000159C110
:105D700072F173EC08F00101222B000109EF2EF003
:105D8000000E81BA010E000AD8A482EF2FF0010E96
:105D90000101226F0001010122510208D8B003D095
:105DA000000182EF2FF0000122C15BF104EC0DF045
:105DB0000101306B2F6B000102C02EF101C02DF1EB
:105DC0000101216B0001010121511F08D8B003D04E
:105DD000000131EF2FF0000130C134F12FC133F158
:105DE0002EC132F12DC131F1390E01012125E96EAB
:105DF000010EEA6ED8B0EA2A000134C15FF133C166
:105E00005EF132C15DF131C15CF1010121515B6F85
:105E1000D8A403D000011CEF2FF00001D89001019D
:105E20005F335E335D335C335B2F02D004D00001FF
:105E300000010EEF2FF0000101015C51010B006E1B
:105E40005D51000B016E5E51000B026E5F51000B45
:105E5000036E000100C0EFFF0101212B0001E3EF01
:105E60002EF001013A53D8A403D000013CEF2FF0EB
:105E70000001310E3DEF2FF0300E0101596F00018E
:105E800059C172F173EC08F001013B53D8A403D05F
:105E900000014FEF2FF00001310E50EF2FF0300EC8
:105EA0000101596F000159C172F173EC08F0010151
:105EB0003C53D8A403D0000162EF2FF00001310E53
:105EC00063EF2FF0300E0101596F000159C172F1DB
:105ED00073EC08F001014153D8A403D0000175EF21
:105EE0002FF00001310E76EF2FF0300E0101596FC7
:105EF000000159C172F173EC08F00101222B00017D
:105F0000CBEF2EF088EF39F0010124510C08D8B402
:105F100003D00001A5EF2FF00001060EA96EA86ABC
:105F2000A69CA69EA684F250006EF29E0F01550E0E
:105F3000A76EAA0EA76EA6820001A6B29DEF2FF053
:105F4000A6940050F21288EF39F0010124510D0897
:105F5000D8B403D00001C3EF30F00001010E926EFF
:105F60000101216B0001010121511208D8B003D0B9
:105F70000001D6EF2FF00001390E01012125016E3D
:105F8000010E036ED8B0032A0150596F000103C0FF
:105F90005AF12EEC26F05AC1EAFF59C1E9FF01C0BF
:105FA000EFFF0101212B0001B3EF2FF0040E0101DF
:105FB000226F0001010122510708D8B003D000016F
:105FC00048EF30F0000122C15BF104EC0DF002C09B
:105FD0002AF101C029F101012951F00B596F2A5111
:105FE0005A6F2251030DF350F60F390FE96E010E6F
:105FF000EA6ED8B0EA2AEF50080DF35059255E6FCB
:10600000000E5A215F6F2251030DF350F50F390F27
:10601000E96E010EEA6ED8B0EA2AEF50040DF35093
:106020005E25636F000E5F21646F2251030DF350F4
:10603000F40F390FE96E010EEA6ED8B0EA2AD89053
:10604000EF34006E6325686F000E6421696F29517B
:10605000010B006E2A51000B036E005068252B6F58
:10606000035069212C6F000181EC03F02CC159F120
:1060700001015A6B000122C160F159C161F12BC1CC
:1060800062F1D7EC03F00101222B0001DAEF2FF0CF
:10609000000E81BA010E000AD8A4C1EF30F0010E43
:1060A0000101226F0001010122510208D8B003D082
:1060B0000001C1EF30F0000122C15BF104EC0DF0F2
:1060C00002C02AF101C029F101012951F00B596FD9
:1060D0002A515A6F2251030DF3500B0F390FE96EFD
:1060E000010EEA6ED8B0EA2AEF50080DF350592598
:1060F0005E6F000E5A215F6F2251030DF3500A0F9D
:10610000390FE96E010EEA6ED8B0EA2AEF50040D9D
:10611000F3505E25636F000E5F21646F2251030D03
:10612000F350090F390FE96E010EEA6ED8B0EA2A72
:10613000D890EF34006E6325686F000E6421696F9C
:106140002951010B006E2A51000B036E0050682587
:106150002B6F035069212C6F000181EC03F02CC1DF
:1061600059F101015A6B000122C160F159C161F17D
:106170002BC162F1D7EC03F00101222B000153EF98
:1061800030F088EF39F0010124510E08D8B403D063
:10619000000158EF31F00001010E926E81EC03F026
:1061A0002EEC26F002C05AF101C059F1080EA96E7A
:1061B00059C1A8FFA69CA69EA684F250006EF29E2E
:1061C0000F01550EA76EAA0EA76EA6820001A6B2F9
:1061D000E7EF30F0A6940050F212080EA96EA69CCC
:1061E000A69EA680A8500108D8A403EF31F0110E96
:1061F0000101606FFF0E616F200E626F0001D7EC2E
:1062000003F056EF31F0110E0101606FFF0E616F68
:10621000626B0001D7EC03F0010E926E81EC03F08B
:10622000010E0101226F0001010122510708D8B0BF
:1062300003D0000156EF31F0000122C15BF104EC04
:106240000DF00101306B2F6B000102C02EF101C077
:106250002DF101012D51E00B296F2E512A6F2D5187
:106260000F0B2B6F2E51000B2C6F2B5129252D6FEF
:106270002C512A212E6F2F6B306B000181EC03F023
:106280002EC15AF12FC15BF130C15CF101015D6B90
:10629000000122C160F15AC161F12DC162F1D7EC58
:1062A00003F00101222B000114EF31F088EF39F0E7
:1062B000010124510F08D8B403D000017BEF31F065
:1062C00000019AEC05F0120EA96EA86AA69CA69E83
:1062D000A684F250006EF29E0F01550EA76EAA0E14
:1062E000A76EA6820001A6B273EF31F0A69400500B
:1062F000F21288EF39F0010124511008D8B403D00C
:10630000000194EF31F00001090EA96EA69CA69E33
:10631000A680A8500101596F686B000159C167F14F
:1063200064EC11F088EF39F0010124511108D8B460
:1063300003D00001BCEF31F000012EEC26F002C0CA
:106340005AF101C059F1090EA96E59C1A8FFA69CC6
:10635000A69EA684F250006EF29E0F01550EA76E07
:10636000AA0EA76EA6820001A6B2B4EF31F0A694E1
:106370000050F21288EF39F0010124511208D8B40C
:1063800003D00001E5EF31F00001120EA96EA69CCA
:10639000A69EA680A850000AD8A4E3EF31F0010120
:1063A000596B000101015951000167EC00F000092F
:1063B000D8B4E3EF31F00101592B726F000173EC97
:1063C00008F0D2EF31F088EF39F0010124511308C1
:1063D000D8B403D000010EEF32F00001120EA96E06
:1063E000A69CA69EA680A850000AD8B40CEF32F056
:1063F0000101596B000101015951000167EC00F0E6
:106400000009D8B40CEF32F00101592B726F000172
:1064100073EC08F0FBEF31F088EF39F00101245103
:106420001408D8B403D0000136EF32F000012EEC8E
:1064300026F002C05AF101C059F1120EA96E59C1DD
:10644000A8FFA69CA69EA684F250006EF29E0F01A5
:10645000550EA76EAA0EA76EA6820001A6B22EEF59
:1064600032F0A6940050F21288EF39F00101245165
:106470001508D8B403D000011BEF33F00001010E62
:10648000926E090EA96EA69CA69EA680A850120F19
:1064900001015A6F00015AC15BF104EC0DF00101DA
:1064A000306B2F6B000102C02EF101C02DF10101F4
:1064B000216B0001010121510F08D8B003D0000168
:1064C000A8EF32F0000130C134F12FC133F12EC1F9
:1064D00032F12DC131F1390E01012125E96E010E94
:1064E000EA6ED8B0EA2A000134C15FF133C15EF12F
:1064F00032C15DF131C15CF1010121515B6FD8A462
:1065000003D0000193EF32F00001D89001015F3316
:106510005E335D335C335B2F02D004D00001000199
:1065200085EF32F0000101015C51010B006E5D51FD
:10653000000B016E5E51000B026E5F51000B036E8B
:10654000000100C0EFFF0101212B00015AEF32F0E2
:10655000030E0101216F0001010121510608D8B08D
:1065600003D00001D4EF32F00001390E01012125E2
:10657000E96E010EEA6ED8B0EA2AEF52D8A403D031
:106580000001C7EF32F00001310EC8EF32F0300EDB
:106590000101596F000159C172F173EC08F001015A
:1065A000212B0001ACEF32F0000E81BA010E000A7F
:1065B000D8A406EF33F00101216B00010101215144
:1065C0000108D8B003D0000106EF33F00001390E06
:1065D00001012125E96E010EEA6ED8B0EA2AEF52D8
:1065E000D8A403D00001F9EF32F00001310EFAEF28
:1065F00032F0300E0101596F000159C172F173EC94
:1066000008F00101212B0001DEEF32F001014053BF
:10661000D8A403D0000111EF33F00001310E12EFC6
:1066200033F0300E0101596F000159C172F173EC62
:1066300008F088EF39F0010124511608D8B403D0CE
:1066400000014FEF33F000010101216B0001010156
:1066500021510408D8B003D0000149EF33F0000104
:10666000320E01012125E96EEA6AD8B0EA2A00015A
:10667000EFCF59F159C15AF1FEEC26F03A0E010163
:10668000726F000173EC08F00101212B000127EF6C
:1066900033F037C05AF1FEEC26F088EF39F00101F3
:1066A00024511B08D8B403D0000177EF33F0000168
:1066B0002EEC26F002C02AF101C029F12EEC26F0C2
:1066C00002C02CF101C02BF1010E926E81EC03F09F
:1066D0002CC159F101015A6B000129C160F159C166
:1066E00061F12BC162F1D7EC03F088EF39F00101C1
:1066F00024511C08D8B403D00001B0EF33F00001DE
:106700000101686B000124C067F164EC11F02E0EEA
:106710000101726F000173EC08F00101686B000168
:1067200023C067F164EC11F02E0E0101726F0001BD
:1067300073EC08F00101686B000122C067F164ECA2
:1067400011F02E0E0101726F000173EC08F00101CF
:10675000686B000121C067F164EC11F088EF39F03B
:10676000010124511D08D8B403D00001E9EF33F032
:1067700000010101686B000128C067F164EC11F0B1
:106780002E0E0101726F000173EC08F00101686BBD
:10679000000127C067F164EC11F02E0E0101726F49
:1067A000000173EC08F00101686B000126C067F17D
:1067B00064EC11F02E0E0101726F000173EC08F011
:1067C0000101686B000125C067F164EC11F088EFEE
:1067D00039F0010124511E08D8B403D000019BEF09
:1067E00034F00001010E926E01012C6B2B6B030E35
:1067F000216F0001010121510608D8B003D000012A
:1068000027EF34F000012EEC26F002C02AF101C07F
:1068100029F12AC103F001012951026E2151006EB4
:10682000D8A403D000011CEF34F00001D890023648
:106830000336002E16EF34F0025001012B270350CF
:106840002C2300010101212B0001FAEF33F0000E8F
:1068500081BA010E000AD8A45EEF34F00101216B69
:106860000001010121510108D8B003D000015EEF01
:1068700034F000012EEC26F002C02AF101C029F10B
:106880002AC103F001012951026E2151006ED8A4E2
:1068900003D0000153EF34F00001D89002360336E4
:1068A000002E4DEF34F0025001012B2703502C2312
:1068B00000010101212B000131EF34F02EEC26F014
:1068C00002C02AF101C029F101012935026E2A35E1
:1068D000036E0236033602360336023603360236BC
:1068E00003360236033602360336800E0216025095
:1068F0002B2703502C23040E2B27FF0E2C230001E3
:1069000081EC03F0090EA96EA69CA69EA680A85055
:10691000120F01015A6F00012CC15BF101015C6B88
:1069200000015AC160F15BC161F12BC162F1D7EC8A
:1069300003F088EF39F0010124512008D8B403D0C6
:106940000001BAEF34F000010101596B00010101AF
:1069500059510001A8EC00F00009D8B4B8EF34F0A8
:106960000101592B726F000173EC08F0A7EF34F0AE
:1069700088EF39F0010124512108D8B403D0000177
:10698000D9EF34F000010101596B000101015951A7
:106990000001BAEC00F00009D8B4D7EF34F00101DF
:1069A000592B726F000173EC08F0C6EF34F088EFDA
:1069B00039F0010124512208D8B403D0000115EFA9
:1069C00035F00001000E81BA010E000AD8A4FFEFD5
:1069D00034F00101596B0001010159510001C7EC6C
:1069E00000F00009D8B4FDEF34F00101592B726FAB
:1069F000000173EC08F0ECEF34F013EF35F0010117
:106A0000596B0001010159510001D5EC00F000095A
:106A1000D8B413EF35F00101592B726F000173ECFC
:106A200008F002EF35F088EF39F001012451230816
:106A3000D8B403D0000134EF35F000010101596BE7
:106A40000001010159510001E3EC00F00009D8B444
:106A500032EF35F00101592B726F000173EC08F031
:106A600021EF35F088EF39F0010124512A08D8B41C
:106A700003D000014DEF35F00001020EA96EA69C77
:106A8000A69EA680A8500101596F686B000159C1EC
:106A900067F164EC11F088EF39F0010124512B0803
:106AA000D8B403D0000166EF35F00001030EA96EE3
:106AB000A69CA69EA680A8500101596F686B000194
:106AC00059C167F164EC11F088EF39F001012451EC
:106AD0002C08D8B403D000017FEF35F00001040E7C
:106AE000A96EA69CA69EA680A8500101596F686B4E
:106AF000000159C167F164EC11F088EF39F0010130
:106B000024512D08D8B403D0000198EF35F00001CE
:106B1000050EA96EA69CA69EA680A8500101596FDD
:106B2000686B000159C167F164EC11F088EF39F02E
:106B3000010124512E08D8B403D00001B1EF35F083
:106B40000001130EA96EA69CA69EA680A850010166
:106B5000596F686B000159C167F164EC11F088EF5F
:106B600039F0010124512F08D8B403D00001CAEF35
:106B700035F00001140EA96EA69CA69EA680A85012
:106B80000101596F686B000159C167F164EC11F0A4
:106B900088EF39F0010124513008D8B403D0000146
:106BA000E3EF35F00001150EA96EA69CA69EA68007
:106BB000A8500101596F686B000159C167F164EC7D
:106BC00011F088EF39F0010124513108D8B403D015
:106BD0000001FCEF35F00001160EA96EA69CA69EE2
:106BE000A680A8500101596F686B000159C167F177
:106BF00064EC11F088EF39F0010124513208D8B467
:106C000003D0000115EF36F00001170EA96EA69C07
:106C1000A69EA680A8500101596F686B000159C15A
:106C200067F164EC11F088EF39F001012451330869
:106C3000D8B403D000012EEF36F00001180EA96E73
:106C4000A69CA69EA680A8500101596F686B000102
:106C500059C167F164EC11F088EF39F0010124515A
:106C60003408D8B403D0000147EF36F00001190E04
:106C7000A96EA69CA69EA680A8500101596F686BBC
:106C8000000159C167F164EC11F088EF39F001019E
:106C900024513508D8B403D0000160EF36F000016C
:106CA0001A0EA96EA69CA69EA680A8500101596F37
:106CB000686B000159C167F164EC11F088EF39F09D
:106CC000010124513608D8B403D0000174EF37F025
:106CD0000001010E926E81EC03F001015A6B1B0E54
:106CE000596F00010DEC27F002C05AF101C059F1B3
:106CF00059C15BF104EC0DF00101306B2F6B000109
:106D000002C02EF101C02DF10A0E0101216F000118
:106D1000010121510D08D8B003D00001D6EF36F0A3
:106D2000000130C134F12FC133F12EC132F12DC138
:106D300031F1390E01012125E96E010EEA6ED8B05C
:106D4000EA2A000134C15FF133C15EF132C15DF165
:106D500031C15CF1010121515B6FD8A403D0000166
:106D6000C1EF36F00001D89001015F335E335D332F
:106D70005C335B2F02D004D000010001B3EF36F08A
:106D8000000101015C51010B006E5D51000B016EB1
:106D90005E51000B026E5F51000B036E000100C0DC
:106DA000EFFF0101212B000188EF36F001015A6B42
:106DB0001B0E596F00017CEC27F002C05AF101C094
:106DC00059F159C15BF104EC0DF00101306B2F6BEF
:106DD000000102C02EF101C02DF11B0EA96EA69C70
:106DE000A69EA680A8500108D8B415EF37F01B0E58
:106DF000A96EA69CA69EA680A8500308D8B415EF3D
:106E000037F01B0EA96EA69CA69EA680A850060869
:106E1000D8B415EF37F01B0EA96EA69CA69EA680CF
:106E2000A8500708D8A420EF37F02EC12DF12FC1AC
:106E30002EF130C12FF10101306B000128EF37F046
:106E4000000E01012E17000E2F17000E3017000143
:106E500001012D372E372F3730372D372E372F376B
:106E600030372D372E372F3730372D372E372F37F6
:106E70003037F00E2D174651080DF3502D25596F60
:106E8000000E2E215A6F000E2F215B6F000E302155
:106E90005C6F4551040DF35059255D6F000E5A216A
:106EA0005E6F000E5B215F6F000E5C21606FD890FB
:106EB0004435006E5D25616F000E5E21626F000E2D
:106EC0005F21636F000E6021646F43516125656F20
:106ED000000E6221666F000166C168F165C167F14D
:106EE00064EC11F088EF39F0010124513708D8B46F
:106EF00003D000018DEF37F000011B0EA96EA69C98
:106F0000A69EA680A8500101596F686B000159C167
:106F100067F164EC11F088EF39F001012451380871
:106F2000D8B403D00001B5EF37F000012EEC26F005
:106F300002C05AF101C059F11B0EA96E59C1A8FF38
:106F4000A69CA69EA684F250006EF29E0F01550EDE
:106F5000A76EAA0EA76EA6820001A6B2ADEF37F00B
:106F6000A6940050F21288EF39F00101245139083B
:106F7000D8B403D00001F8EF38F00001010E926E92
:106F80002EEC26F001C045F11B0EA96EA69CA69E14
:106F9000A680A8500808D8B4D8EF37F0080EA96E1C
:106FA000A69CA69EA680A850000AD8A4DBEF37F0C6
:106FB0000101456B00012EEC26F002C02AF101C050
:106FC00029F101012A53D8B403D00001F2EF37F0C0
:106FD0000001010129510008D8A003D00001F6EFFB
:106FE00038F0000101012A510F08D8B003D0000188
:106FF000F6EF38F000012AC12CF129C12BF1010173
:107000002B510F0B596F2C51000B5A6F2B6B5935AD
:107010002C6F2C37FC0E2C175A6B1B0E596F00016E
:107020000DEC27F002C05AF101C059F159C15BF1D2
:1070300004EC0DF00101306B2F6B000102C02EF14A
:1070400001C02DF101012D99C30E2E17000E2F172F
:10705000000E30172B512D25596F2C512E215A6FB0
:10706000000E2F215B6F000E30215C6F4539006EE2
:10707000F00E0016005059252D6F000E5A212E6F6C
:10708000000E5B212F6F000E5C21306F000181EC40
:1070900003F001015A6B1B0E596F00010DEC27F034
:1070A00002C05AF101C059F12EC15CF12FC15DF14E
:1070B00030C15EF101015F6B000159C160F15CC13B
:1070C00061F12DC162F1D7EC03F02AC12CF129C185
:1070D0002BF101012C332B332C332B332C332B335B
:1070E0002C332B330F0E2C171B0EA96EA69CA69EBD
:1070F000A680A8500108D8A403D000019FEF38F063
:1071000000011B0EA96EA69CA69EA680A85003088F
:10711000D8B49FEF38F01B0EA96EA69CA69EA68041
:10712000A8500608D8B49FEF38F01B0EA96EA69C95
:10713000A69EA680A8500708D8A4C9EF38F0010180
:107140005A6B1B0E596F00017CEC27F002C05AF1FC
:1071500001C059F159C15BF104EC0DF002C02AF1F4
:1071600001C029F181EC03F001015A6B1B0E596F2C
:1071700000017CEC27F002C05AF101C059F159C15D
:1071800060F12BC161F129C162F1D7EC03F0F6EF98
:1071900038F001015A6B1B0E596F00017CEC27F08F
:1071A00002C05AF101C059F159C15BF104EC0DF074
:1071B00002C02AF101C029F181EC03F001015A6BF0
:1071C0001B0E596F00017CEC27F002C05AF101C080
:1071D00059F12AC15BF101015C6B000159C160F1F9
:1071E0005BC161F12BC162F1D7EC03F088EF39F09C
:1071F000010124513A08D8B403D0000182EF39F0DC
:107200000001010E926E81EC03F001015A6B1B0E1E
:10721000596F00010DEC27F002C05AF101C059F17D
:1072200059C15BF104EC0DF00101306B2F6B0001D3
:1072300002C02EF101C02DF10101216B00010101FD
:1072400021510F08D8B003D000016DEF39F00001D3
:1072500030C134F12FC133F12EC132F12DC131F1E2
:10726000390E01012125E96E010EEA6ED8B0EA2A35
:10727000000134C15FF133C15EF132C15DF131C152
:107280005CF1010121515B6FD8A403D0000158EFDC
:1072900039F00001D89001015F335E335D335C3318
:1072A0005B2F02D004D0000100014AEF39F0000149
:1072B00001015C51010B006E5D51000B016E5E51CE
:1072C000000B026E5F51000B036E000100C0EFFF68
:1072D0000101212B00011FEF39F001013D53D8A41A
:1072E00003D0000178EF39F00001310E79EF39F069
:1072F000300E0101596F000159C172F173EC08F0B1
:1073000088EF39F03F0E0101726F000173EC08F055
:107310008EEF39F023C172F173EC08F0F2EF28F030
:10732000E5EF27F0010E016E98EF39F0000E016EC7
:1073300050EF3CF0080EAD6FAC6B2990C3C02AF043
:10734000C4C02BF0B8C025F1B7C024F16DEC14F027
:10735000BAC025F1B9C024F16DEC14F00101256B20
:10736000CA0E246F000101EC14F00101256BC60E5A
:10737000246F000101EC14F001012251020B000AFC
:10738000D8A403D00001C9EF39F00001600ECAEFA4
:1073900039F0500E0101236F000123C172F173EC2B
:1073A00008F022C172F173EC08F00B0E0101726F4C
:1073B000000173EC08F0B80E0101726F000173EC6C
:1073C00008F001012251020B000AD8A403D00001E9
:1073D0000DEF3AF000010101256B280E246F00012A
:1073E000D8EC13F0020E0101726F000173EC08F08B
:1073F000040E0101726F000173EC08F0050E01012B
:10740000256FB40E246F00016DEC14F00101256BA3
:10741000240E246F0001D8EC13F00101256B190E26
:10742000246F000178EC14F00101256BB30E246F7A
:10743000000178EC14F00101736B00014CEC08F0D2
:10744000060E0101736F00014CEC08F0140EC15DD3
:107450000101236F000E0001C2590101246F0001D8
:1074600024C126F123C125F10DEC15F02A500101AC
:10747000236F231F000123C172F173EC08F02B501E
:107480000101236F231F000123C172F173EC08F087
:107490000101256B246B00016DEC14F001012251F8
:1074A000020B000AD8A403D000015FEF3AF00001FC
:1074B0000101256B2C0E246F0001D8EC13F093EF23
:1074C0003AF021EC08F02AC0C3F02BC0C4F06E5291
:1074D000D8A473EF3AF06D502708D8A073EF3AF0B4
:1074E0006E6A280E6D6E01012151020B000AD8A4AC
:1074F00003D0000181EF3AF00001040E6D26000E6A
:107500006E226EC0C2F06DC0C1F00101256B246B0C
:107510000001D8EC13F0060EAE6FAFEC14F021C1F1
:1075200022F19AEF39F06CEC15F060EF3CF0100EA0
:1075300001011E6F29902B6A00012BC02AF0010166
:10754000236BB90E226F0001A4EC1AF00152D8B4DB
:1075500064EF3CF00101236BB70E226F0001A4EC35
:107560001AF00152D8B464EF3CF00101226BC60E50
:10757000216F0001E1EC1AF00152D8B464EF3CF045
:107580000101226BCA0E216F0001E1EC1AF00152D9
:10759000D8B464EF3CF0010E01016C6F1C0E6B6FF0
:1075A000000188EC0BF00152D8B464EF3CF0010EFE
:1075B00001016C6F1D0E6B6F000188EC0BF0015226
:1075C000D8B464EF3CF00101236B060E226F00017A
:1075D00030EC1BF00152D8B464EF3CF0C253D8A495
:1075E000F7EF3AF0C1512708D8B064EF3CF01950DA
:1075F000AF5DD8A464EF3CF01A50B05DD8A464EF3E
:107600003CF01B50B15DD8A464EF3CF01C50B25D5F
:10761000D8A464EF3CF0140EC15D0101216F000E8F
:107620000001C2590101226F000122C126F121C1CE
:1076300025F10DEC15F00101256B190E246F0001E9
:1076400078EC14F00101256BB30E246F000178EC87
:1076500014F00101736B00014CEC08F0060E0101FF
:10766000736F00014CEC08F001011C515008D8A0C8
:1076700003D000015AEF3BF00001C153D8A445EFFD
:107680003BF0C253D8B45AEF3BF00101236B040E18
:10769000226F000130EC1BF00152D8B45AEF3BF0DE
:1076A000040EC15F000EC25B100E01011C5F0001E1
:1076B00034EF3BF0280EC15DD06F000EC259D16F80
:1076C0003FC020F13EC01FF1D1C023F1D0C022F154
:1076D00030EC1BF020C123F11FC122F1BEEC1DF0E4
:1076E0002A3C64EF3CF02B3C64EF3CF00101216B41
:1076F00000016EEC1AF00101256B280E246F0001C9
:10770000D8EC13F0C46BC4C0C3F02996299429881F
:1077100001011D51040B000AD8A403D0000197EF0A
:107720003BF0000101011E6B000154EF3CF0010130
:107730001D51020B000AD8A403D00001D6EF3BF084
:1077400000010101246BC60E236F266B010E256F0D
:10775000000173EC22F0B7510D08D8A4B4EF3BF050
:10776000B853D8B4BDEF3BF0B7515008D8A4D0EF10
:107770003BF0B853D8A4D0EF3BF0FF0ECB6FFF0E19
:10778000CA6FCF51036ECE51CE2BD8B4CF2BCC6F56
:1077900003C0CDF0120E01011E6F0001D4EF3BF0CB
:1077A000140E01011E6F000154EF3CF001011D5148
:1077B000010B000AD8A403D00001F5EF3BF0000153
:1077C000010ED0250101216F000E0001D121010120
:1077D000226F246BC60E236F000122C126F121C146
:1077E00025F173EC22F054EF3CF001011D51100B18
:1077F000000AD8A403D0000154EF3CF00001D0519E
:10780000D111D8B411EF3CF00101246BC60E236FE7
:107810000001D1C026F1D0C025F173EC22F014EFA5
:107820003CF001011E6B0001B7510D08D8A440EFD8
:107830003CF0B853D8A440EF3CF0CA53D8A440EF72
:107840003CF0CB53D8A440EF3CF00101216B000188
:1078500001012151000130EC00F00101212B716F79
:1078600000019FEC08F00C0E0101215DD8B403D09B
:10787000000128EF3CF0110E1E6F000154EF3CF0A8
:10788000B7515008D8A454EF3CF0B853D8A454EFE3
:107890003CF0D051D111D8B454EF3CF0F6EF27F0C2
:1078A000110E01011E6F000101011E53D8A403D067
:1078B000000160EF3CF000011EC121F161EF3AF0E0
:1078C000010E016E66EF3CF0000E016E85EF3FF099
:1078D000F86AD08EFE0E006E050E016EEA6A020E88
:1078E000E96EEF6AE92AD8B4EA2A002E71EF3CF07B
:1078F000012E71EF3CF0EA6AE96A070EC16E056A73
:10790000066A010E076E086A096A0A6A0B6A810E26
:10791000AF6E260EAC6E900EAB6E156A166A050E33
:10792000186E326A400E336EF60E346EFD0E356EF2
:10793000366A376AC56BEC6B0101196B1A6B000173
:10794000F29CF29EF2BEA1EF3CF0130E926E826AA0
:10795000FF0E946EFF0E956E8480848284849690D0
:1079600096929694000E80B8010E000AD8A426EFD5
:107970003DF0140E01011C6F0001FA0E0101686F49
:107980000001C6EC01F001011C2F02D003D0000160
:107990000001F3D7000E80B8010E000AD8B403D05E
:1079A000000126EF3DF00001A96AA69CA69EA680D4
:1079B000A850366E010EA96EA69CA69EA680A85061
:1079C000376E01011F6B190E1E6FC00E206FA80EBF
:1079D000216F226B020E236F0001DCEC01F001012C
:1079E0001F6B210E1E6FFF0E206FFF0E216FFF0E0B
:1079F000226F236B0001DCEC01F001011F6B250EEF
:107A00001E6FC00E206FA80E216F226B010E236F18
:107A10000001DCEC01F024EC02F0120EA96E010E64
:107A2000A86EA69CA69EA684F250006EF29E0F0140
:107A3000550EA76EAA0EA76EA6820001A6B21EEF73
:107A40003DF0A6940050F2129AEC05F0F19ECF6A38
:107A5000B50ECD6ECD9E0101256B120E246F276BE6
:107A6000266B000136EC07F01486149A1498808473
:107A70008086298629842998FE0E946E8B808B90AF
:107A80001E0E0101686F0001C6EC01F0640E0101D9
:107A9000686F0001C6EC01F08B801E0E0101686F5B
:107AA0000001C6EC01F0FF0E946E01011C6B000199
:107AB00001011C5100011CEC01F001011C2B000113
:107AC0009EA860EF3DF0AD6E040E01011C5DD8B4C0
:107AD00003D0000158EF3DF0000E81BA010E000AFC
:107AE000D8B403D0000190EF3DF0000101011C6B00
:107AF000000101011C510001C7EC00F001011C2B29
:107B000000019EA881EF3DF0AD6E0A0E01011C5DE3
:107B1000D8B403D0000179EF3DF00001A8EF3DF0AB
:107B200001011C6B000101011C510001D5EC00F0AA
:107B300001011C2B00019EA89BEF3DF0AD6E0A0ECB
:107B400001011C5DD8B403D0000193EF3DF00001AA
:107B5000200E0101716F00019FEC08F001011C6B08
:107B6000000101011C51000127EC01F001011C2B57
:107B7000716F00019FEC08F00F0E01011C5DD8B47D
:107B800003D00001B1EF3DF0030E1D6F0001390E6F
:107B90000101716F00019FEC08F001011D2F02D05F
:107BA00004D000010001C7EF3DF0200E716F00010D
:107BB0009FEC08F001011C6B000101011C51000148
:107BC000BAEC00F001011C2B716F00019FEC08F072
:107BD000090E01011C5DD8B403D00001DDEF3DF0BA
:107BE0000A0E716F00019FEC08F0BFEC08F0015223
:107BF000D8A473EF3EF001011C6B000101011C5180
:107C0000000137EC01F001011C2B716F00019FECAA
:107C100008F0070E01011C5DD8B403D00001FEEF8F
:107C20003DF0000196EF0CF00A0EA96E310EA86E21
:107C3000A69CA69EA684F250006EF29E0F01550EE1
:107C4000A76EAA0EA76EA6820001A6B225EF3EF08F
:107C5000A6940050F2120B0EA96E320EA86EA69CCE
:107C6000A69EA684F250006EF29E0F01550EA76EDE
:107C7000AA0EA76EA6820001A6B23CEF3EF0A69423
:107C80000050F2120C0EA96E330EA86EA69CA69E92
:107C9000A684F250006EF29E0F01550EA76EAA0E3A
:107CA000A76EA6820001A6B253EF3EF0A694005044
:107CB000F212120EA96EA86AA69CA69EA684F25085
:107CC000006EF29E0F01550EA76EAA0EA76EA68239
:107CD0000001A6B269EF3EF0A6940050F2129AECB1
:107CE00005F0F5EF3DF0A8EF0EF0F5EC0FF0120EF9
:107CF000A96EA69CA69EA680A850176E1752D8A45F
:107D000088EF3EF01C6A1B6A1A6A196A93EF3EF00C
:107D1000148EBFEC08F0B8EC11F000EC12F048EC57
:107D200012F0CAEC12F00D0E9EA894EF3EF0AD6E6C
:107D30000A0E9EA899EF3EF0AD6E090EA96E020ED6
:107D4000A86EA69CA69EA684F250006EF29E0F011D
:107D5000550EA76EAA0EA76EA6820001A6B2AEEFC0
:107D60003EF0A6940050F2121B0EA96E010EA86EF2
:107D7000A69CA69EA684F250006EF29E0F01550EA0
:107D8000A76EAA0EA76EA6820001A6B2C5EF3EF0AE
:107D9000A6940050F212000E80B8010E000AD8A47A
:107DA0000BEF3FF00D0E9EA8D3EF3EF0AD6E0A0E26
:107DB0009EA8D8EF3EF0AD6E01011B6B00010101E2
:107DC0001B513F08D8B003D000010AEF3FF000017B
:107DD0001BC15BF104EC0DF002C01DF101C01CF1F0
:107DE0001DC123F1370E0101246F000190EC12F048
:107DF0001CC123F1370E0101246F000190EC12F039
:107E0000200E9EA801EF3FF0AD6E01011B2B00017B
:107E1000DFEF3EF08088ADEC09F01752D8A418EFE0
:107E20003FF01850165CD8B018EF3FF0EAEF17F0AB
:107E30001752D8A448EF3FF01850165CD8A048EF6E
:107E40003FF0148E1952D8A434EF3FF01A52D8A440
:107E500034EF3FF01B52D8A434EF3FF01C52D8A4AB
:107E600034EF3FF0BFEC08F0B8EC11F000EC12F08A
:107E700048EC12F0CAEC12F0166AF4C0F2F0F3C04B
:107E8000F1F0EC510308D8A448EF3FF0010EEC6F7D
:107E900070EF19F00152D8B487EF3FF00101216B68
:107EA00000016EEC1AF0AC510608D8A45FEF3FF069
:107EB000AD510808D8A45FEF3FF019EF1CF0AC53A8
:107EC000D8A485EF3FF0AD510808D8A485EF3FF066
:107ED0002FEF1DF00152D8B485EF3FF0AE2D75EFB6
:107EE0003FF072EF1EF085EF3FF0AE511108D8A4BD
:107EF0007EEF3FF076EF21F085EF3FF0AE510608C0
:107F0000D8A485EF3FF097EF3AF03D6A3C6A152C14
:0C7F10008BEF3FF0FF00CBEF3EF00300D2
:020000040030CA
:0C000000FFFAFCFEFFFFFBFFFFFFFFFF0D
:00000001FF
